:020000040000FA
:0408000088EF0BF082
:1008100003B273EF05F0F2B491EF05F09EB099EFDB
:1008200005F09EB2A1EF05F0F2A81AEF04F0F2B2C3
:1008300021EF04F0F2B01FEF04F037EF0BF0F29667
:10084000F290CD90F2929EA02BEF04F00101533F65
:100850002BEF04F0542BB2C1B6F1B3C1B7F1B4C160
:10086000B8F1B5C1B9F1AEC1B2F1AFC1B3F1B0C128
:10087000B4F1B1C1B5F1AAC1AEF1ABC1AFF1ACC138
:10088000B0F1ADC1B1F1A6C1AAF1A7C1ABF1A8C148
:10089000ACF1A9C1ADF1A2C1A6F1A3C1A7F1A4C158
:1008A000A8F1A5C1A9F19EC1A2F19FC1A3F1A0C168
:1008B000A4F1A1C1A5F19AC19EF19BC19FF19CC178
:1008C000A0F19DC1A1F1CECF9AF1CFCF9BF153C141
:1008D0009CF154C19DF1CF6ACE6A0101536B546BF8
:1008E0009E90CD800FBC0F8E0FBA7AEF04F00F8A66
:1008F00037EF0BF013880F8C0FBEB7EF04F09AC1DF
:100900009EF19BC19FF19CC1A0F19DC1A1F19EC12F
:10091000A2F19FC1A3F1A0C1A4F1A1C1A5F1A2C1FF
:10092000A6F1A3C1A7F1A4C1A8F1A5C1A9F1A6C1CF
:10093000AAF1A7C1ABF1A8C1ACF1A9C1ADF1AAC19F
:10094000AEF1ABC1AFF1ACC1B0F1ADC1B1F1AEC16F
:10095000B2F1AFC1B3F1B0C1B4F1B1C1B5F1B2C13F
:10096000B6F1B3C1B7F1B4C1B8F1B5C1B9F1010184
:100970005E6B5F6B606B616B9A515E279B515F236F
:100980009C5160239D5161239E515E279F515F239F
:10099000A0516023A1516123A2515E27A3515F237F
:1009A000A4516023A5516123A6515E27A7515F235F
:1009B000A8516023A9516123AA515E27AB515F233F
:1009C000AC516023AD516123AE515E27AF515F231F
:1009D000B0516023B1516123B2515E27B3515F23FF
:1009E000B4516023B5516123B6515E27B7515F23DF
:1009F000B8516023B9516123D8900101613360334C
:100A00005F335E33D8900101613360335F335E330F
:100A1000D8900101613360335F335E3300C10CF164
:100A200001C10DF102C10EF103C10FF104C110F1BA
:100A300005C111F106C112F107C113F108C114F18A
:100A400009C115F10AC116F10BC117F134C135F115
:100A500011B836EF05F00101620E046F010E056F4B
:100A6000000E066F000E076F3FEF05F00101A70EA5
:100A7000046F020E056F000E066F000E076F5EC159
:100A800000F15FC101F160C102F161C103F155ECF8
:100A90002FF003BF04D01CBE02D01CA0108C11A0EC
:100AA00057EF05F010BA57EF05F00F80108A0CC110
:100AB00000F10DC101F10EC102F10FC103F110C12E
:100AC00004F111C105F112C106F113C107F114C1FE
:100AD00008F115C109F116C10AF117C10BF135C1B1
:100AE00034F137EF0BF00392ABB2AB98AB88030154
:100AF00003EE00F080517F0BE92604C0EFFF802B4E
:100B00008151805D700BD8A48B8200008051815D83
:100B1000700BD8A48B9281518019D8B4079037EF0D
:100B20000BF0F2940101453F37EF0BF0462B37EF06
:100B30000BF09E900101533F37EF0BF0542B37EF32
:100B40000BF09E9211B839EF08F0040066A1A9EFEE
:100B500005F08BB4B3EF05F010ACB3EF05F08B8468
:100B6000109CB4EF05F08B94077C07ACCFEF05F039
:100B7000C274C2B4C9EF05F0C3CFB7F5C4CFB8F59E
:100B80000501D890B833B733D890B833B733D0EF26
:100B900005F0C3CF55F1C4CF56F1D0EF05F0C282B6
:100BA00007B442EF06F047C14BF148C14CF149C1CF
:100BB0004DF14AC14EF15EC162F15FC163F160C1A6
:100BC00064F161C165F113A8E8EF05F0138C139887
:100BD0009AC1BAF19BC1BBF19CC1BCF19DC1BDF1F1
:100BE0009EC1BEF19FC1BFF1A0C1C0F1A1C1C1F1C1
:100BF000A2C1C2F1A3C1C3F1A4C1C4F1A5C1C5F191
:100C0000A6C1C6F1A7C1C7F1A8C1C8F1A9C1C9F160
:100C1000AAC1CAF1ABC1CBF1ACC1CCF1ADC1CDF130
:100C2000AEC1CEF1AFC1CFF1B0C1D0F1B1C1D1F100
:100C3000B2C1D2F1B3C1D3F1B4C1D4F1B5C1D5F1D0
:100C4000B6C1D6F1B7C1D7F1B8C1D8F1B9C1D9F1A0
:100C5000B7C5B9F5B8C5BAF5B9C5BBF5BAC5BCF5E0
:100C6000010155515B2756515C23E86A5D230E2E26
:100C700042EF06F05CC157F15DC158F15B6B5C6BF4
:100C80005D6B078E0201002F37EF0BF03C0E006FFB
:100C90001D50E00BE00AE86612881BBE02D01BB4B0
:100CA000108E00C10CF101C10DF102C10EF103C1A2
:100CB0000FF104C110F105C111F106C112F107C114
:100CC00013F108C114F109C115F10AC116F10BC1E4
:100CD00017F134C135F181AA30EF07F037A0EDEFFD
:100CE00006F005012F51000AD8B430EF07F00501D6
:100CF0002F51010AD8B4ACEF06F005012F51020ABA
:100D0000D8B4EDEF06F005012F51030AD8B4EDEF8A
:100D100006F005012F51040AD8B4EDEF06F00501E5
:100D20002F51050AD8B4EDEF06F005012F51060A40
:100D3000D8B4EDEF06F005012F51070AD8B4EDEF56
:100D400006F005012F51320AD8B4AAEF06F02F6B36
:100D500030EF07F030EF07F005015767B7EF06F007
:100D60005867B7EF06F05967B7EF06F05A67BBEF61
:100D700006F030EF07F05BC500F15CC501F15DC521
:100D800002F15EC503F10101010E046F000E056F53
:100D9000000E066F000E076F55EC2FF000C15BF5DB
:100DA00001C15CF502C15DF503C15EF5010100679B
:100DB000E1EF06F00167E1EF06F00267E1EF06F010
:100DC000036730EF07F057C55BF558C55CF559C5AB
:100DD0005DF55AC55EF51AEF07F00FBE02EF07F09A
:100DE00010A007EF07F001014767FEEF06F0486724
:100DF000FEEF06F04967FEEF06F04A6702EF07F0E4
:100E000007EF07F007AE07EF07F01AEF07F005014D
:100E1000312F30EF07F03C0E316F302F30EF07F0FD
:100E20000101000E626FE00E636FA50E646F010E8C
:100E3000656F138800011650000AD8B428EF07F038
:100E400000011650030AD8B42DEF07F030EF07F079
:100E50000001010E166E30EF07F00001040E166E51
:100E60000501666B37B736EF07F066810CC100F1FC
:100E70000DC101F10EC102F10FC103F110C104F166
:100E800011C105F112C106F113C107F114C108F136
:100E900015C109F116C10AF117C10BF135C134F1C1
:100EA00000C10CF101C10DF102C10EF103C10FF13E
:100EB00004C110F105C111F106C112F107C113F10E
:100EC00008C114F109C115F10AC116F10BC117F1DE
:100ED00034C135F101018E6775EF07F08F6775EF4B
:100EE00007F0906775EF07F0916779EF07F0AAEFC9
:100EF00007F092C100F193C101F194C102F195C1D3
:100F000003F10101010E046F000E056F000E066F64
:100F1000000E076F55EC2FF000C192F101C193F163
:100F200002C194F103C195F1010100679FEF07F041
:100F300001679FEF07F002679FEF07F00367AAEFD3
:100F400007F08EC192F18FC193F190C194F191C1DC
:100F500095F10F80D57ED5BE6ED0D6CF47F1D7CFD5
:100F600048F145C149F1E86AE8CF4AF1138A1CBE4D
:100F700002D01CA0108C109047C100F148C101F1B3
:100F800049C102F14AC103F101010A0E046F000ECA
:100F9000056F000E066F000E076F55EC2FF003AFC4
:100FA0001080010154A7E1EF07F00F9A0F9C0F9EEC
:100FB0000101000E5E6F600E5F6F3D0E606F080EE8
:100FC000616F010147BFF1EF07F04867F1EF07F0EC
:100FD0004967F1EF07F04A67F1EF07F0F28816EF83
:100FE00008F0F2985E6B5F6B606B616B9A6B9B6B4A
:100FF0009C6B9D6B9E6B9F6BA06BA16BA26BA36B9D
:10100000A46BA56BA66BA76BA86BA96BAA6BAB6B4C
:10101000AC6BAD6BAE6BAF6BB06BB16BB26BB36BFC
:10102000B46BB56BB66BB76BB86BB96BD76AD66A76
:101030000101456B466B0CC100F10DC101F10EC100
:1010400002F10FC103F110C104F111C105F112C188
:1010500006F113C107F114C108F115C109F116C158
:101060000AF117C10BF135C134F137EF0BF037EF4F
:101070000BF00201002F9BEF0AF0D59ED6CF47F16F
:10108000D7CF48F145C149F1E86AE8CF4AF1138A60
:10109000D76AD66A0101456B466BD58E1D50E00BB1
:1010A000E00AE86612881BBE02D01BB4108E1AAE8E
:1010B0001F8C00C10CF101C10DF102C10EF103C181
:1010C0000FF104C110F105C111F106C112F107C100
:1010D00013F108C114F109C115F10AC116F10BC1D0
:1010E00017F134C135F10FA0109A11B883EF08F051
:1010F0000101620E046F010E056F000E066F000EF7
:10110000076F8CEF08F00101A70E046F020E056F48
:10111000000E066F000E076F47C100F148C101F1D4
:1011200049C102F14AC103F155EC2FF003BF9FEF13
:1011300008F01CBE02D01CA0108C11B00F800CC196
:1011400000F10DC101F10EC102F10FC103F110C197
:1011500004F111C105F112C106F113C107F114C167
:1011600008F115C109F116C10AF117C10BF135C11A
:1011700034F102013C0E006F00C10CF101C10DF110
:1011800002C10EF103C10FF104C110F105C111F14B
:1011900006C112F107C113F108C114F109C115F11B
:1011A0000AC116F10BC117F134C135F181AA15EF4F
:1011B00009F037A060EF09F005012F51000AD8B4FB
:1011C000A3EF09F005012F51010AD8B41FEF09F070
:1011D00005012F51020AD8B460EF09F005012F5123
:1011E000030AD8B460EF09F005012F51040AD8B4FE
:1011F00060EF09F005012F51050AD8B460EF09F03E
:1012000005012F51060AD8B460EF09F005012F51EE
:10121000070AD8B460EF09F005012F51320AD8B49B
:101220001DEF09F02F6BA3EF09F000011650030A20
:10123000D8B460EF09F0A3EF09F0A3EF09F00501BE
:1012400057672AEF09F058672AEF09F059672AEF24
:1012500009F05A672EEF09F0A3EF09F05BC500F122
:101260005CC501F15DC502F15EC503F10101010E2E
:10127000046F000E056F000E066F000E076F55EC31
:101280002FF000C15BF501C15CF502C15DF503C142
:101290005EF50101006754EF09F0016754EF09F0B2
:1012A000026754EF09F00367A3EF09F057C55BF538
:1012B00058C55CF559C55DF55AC55EF58DEF09F069
:1012C0000FBE75EF09F010A07AEF09F00101476732
:1012D00071EF09F0486771EF09F0496771EF09F0A4
:1012E0004A6775EF09F07AEF09F007AE7AEF09F077
:1012F0008DEF09F00501312FA3EF09F03C0E316F9E
:10130000302FA3EF09F00101000E626FE00E636F52
:10131000A50E646F010E656F138800011650000A58
:10132000D8B49BEF09F000011650030AD8B4A0EF1F
:1013300009F0A3EF09F00001010E166EA3EF09F00A
:101340000001040E166E0501666B37B7A9EF09F0B0
:1013500066810CC100F10DC101F10EC102F10FC196
:1013600003F110C104F111C105F112C106F113C15D
:1013700007F114C108F115C109F116C10AF117C12D
:101380000BF135C134F100C10CF101C10DF102C105
:101390000EF103C10FF104C110F105C111F106C135
:1013A00012F107C113F108C114F109C115F10AC105
:1013B00016F10BC117F134C135F101018E67E8EF69
:1013C00009F08F67E8EF09F09067E8EF09F091679F
:1013D000ECEF09F01DEF0AF092C100F193C101F1A9
:1013E00094C102F195C103F10101010E046F000ED9
:1013F000056F000E066F000E076F55EC2FF000C151
:1014000092F101C193F102C194F103C195F101017F
:10141000006712EF0AF0016712EF0AF0026712EF9D
:101420000AF003671DEF0AF08EC192F18FC193F1AC
:1014300090C194F191C195F10F80109047C100F1D6
:1014400048C101F149C102F14AC103F101010A0E8B
:10145000046F000E056F000E066F000E076F55EC4F
:101460002FF003AF1080010154A743EF0AF00F9A49
:101470000F9C0F9E0101000E5E6F600E5F6F3D0EB0
:10148000606F080E616F47C100F148C101F149C1A9
:1014900002F14AC103F10101140E046F050E056F3C
:1014A000000E066F000E076F55EC2FF003AF5CEFD8
:1014B0000AF0F28881EF0AF0F2985E6B5F6B606B66
:1014C000616B9A6B9B6B9C6B9D6B9E6B9F6BA06B18
:1014D000A16BA26BA36BA46BA56BA66BA76BA86B90
:1014E000A96BAA6BAB6BAC6BAD6BAE6BAF6BB06B40
:1014F000B16BB26BB36BB46BB56BB66BB76BB86BF0
:10150000B96B0CC100F10DC101F10EC102F10FC1A7
:1015100003F110C104F111C105F112C106F113C1AB
:1015200007F114C108F115C109F116C10AF117C17B
:101530000BF135C134F104008BB4A6EF0AF010AC06
:10154000A6EF0AF08B84109CA7EF0AF08B94077C1F
:1015500007ACC2EF0AF0C274C2B4BCEF0AF0C3CF4A
:10156000B7F5C4CFB8F50501D890B833B733D890E4
:10157000B833B733C3EF0AF0C3CF55F1C4CF56F138
:10158000C3EF0AF0C28207B435EF0BF047C14BF14D
:1015900048C14CF149C14DF14AC14EF15EC162F101
:1015A0005FC163F160C164F161C165F113A8DBEF54
:1015B0000AF0138C13989AC1BAF19BC1BBF19CC17C
:1015C000BCF19DC1BDF19EC1BEF19FC1BFF1A0C1E3
:1015D000C0F1A1C1C1F1A2C1C2F1A3C1C3F1A4C1B3
:1015E000C4F1A5C1C5F1A6C1C6F1A7C1C7F1A8C183
:1015F000C8F1A9C1C9F1AAC1CAF1ABC1CBF1ACC153
:10160000CCF1ADC1CDF1AEC1CEF1AFC1CFF1B0C122
:10161000D0F1B1C1D1F1B2C1D2F1B3C1D3F1B4C1F2
:10162000D4F1B5C1D5F1B6C1D6F1B7C1D7F1B8C1C2
:10163000D8F1B9C1D9F1B7C5B9F5B8C5BAF5B9C5C9
:10164000BBF5BAC5BCF5010155515B2756515C236A
:10165000E86A5D230E2E35EF0BF05CC157F15DC1DA
:1016600058F15B6B5C6B5D6B078E37EF0BF002C064
:10167000E0FF005001C0D8FF1000A6B23DEF0BF014
:101680000CC0A9FF0BC0A8FFA69EA69CA684F29E34
:10169000550EA76EAA0EA76EA682F28EA694A6B2CB
:1016A0004FEF0BF00C2A1200A96EA69EA69CA680F6
:1016B000A8500C2A120004012C0E826FCBEC0EF005
:1016C00050EC30F00C5054EC0BF0E8CF00F10C5023
:1016D00054EC0BF0E8CF01F101AF74EF0BF0010116
:1016E000FF0E026FFF0E036FF3EC2FF0296780EF00
:1016F0000BF00401200E826FCBEC0EF085EF0BF0A7
:1017000004012D0E826FCBEC0EF0FDEC2DF01200DB
:10171000376A076A0F6A106A116A126A136A156AD1
:10172000166A0F010D0EC16E860EC06E030EC26EDC
:101730000F01680E896E130E926E080E8A6EF30EFC
:10174000936E8B6A900E946EC80E54EC0BF0E8CF3B
:10175000E8FF1098E8A0108810A805D00E0E256E9E
:101760008E0E266E04D00F0E256E8F0E266EE8ECC0
:1017700030F0F18EF19EFC0E54EC0BF0E8CF0BF044
:101780000BA011800BA211820BA411840BA811884D
:10179000C90E54EC0BF0E8CF1AF0CA0E54EC0BF063
:1017A000E8CF1BF0CB0E54EC0BF0E8CF1CF0CC0EC6
:1017B00054EC0BF0E8CF1DF0FB0E54EC0BF0E8CF2F
:1017C00038F0CE0E54EC0BF0E8CF14F0CD0E54EC04
:1017D0000BF0E8CF36F01F6A206A0E6A01015B6BDE
:1017E0005C6B5D6B576B586BF29A0101476B486BF2
:1017F000496B4A6B4B6B4C6B4D6B4E6B4F6B506B2D
:10180000516B526B456B466BD76AD66A0F01280E37
:10181000D56EF28A9D90B00ECD6E01015E6B5F6B4E
:10182000606B616B626B636B646B656B666B676B44
:10183000686B696B536B546BCF6ACE6A0F9A0F9CBF
:101840000F9E9D80760ECA6E9D8202013C0E006F37
:10185000CC6A160E54EC0BF0E8CF00F1170E54ECE6
:101860000BF0E8CF01F1180E54EC0BF0E8CF02F1C9
:10187000190E54EC0BF0E8CF03F1010103AF5BEF5D
:101880000CF050EC30F0160E0C6E00C10BF03DEC7D
:101890000BF0170E0C6E01C10BF03DEC0BF0180EA7
:1018A0000C6E02C10BF03DEC0BF0190E0C6E03C177
:1018B0000BF03DEC0BF000C18EF101C18FF102C1C4
:1018C00090F103C191F100C192F101C193F102C104
:1018D00094F103C195F11A0E54EC0BF0E8CF00F12E
:1018E0001B0E54EC0BF0E8CF01F11C0E54EC0BF086
:1018F000E8CF02F11D0E54EC0BF0E8CF03F101012B
:1019000003AFB1EF0CF050EC30F01A0E0C6E00C1CA
:101910000BF03DEC0BF01B0E0C6E01C10BF03DEC1F
:101920000BF01C0E0C6E02C10BF03DEC0BF01D0E0B
:101930000C6E03C10BF03DEC0BF01A0E54EC0BF0E7
:10194000E8CF00F11B0E54EC0BF0E8CF01F11C0EB8
:1019500054EC0BF0E8CF02F11D0E54EC0BF0E8CF85
:1019600003F100C196F101C197F102C198F103C1E1
:1019700099F1240EAC6E900EAB6E240EAC6E080E78
:10198000B86E000EB06E1F0EAF6E0401806B816BDF
:101990000F01900EAB6E0F019D8A0301806B816B6E
:1019A000C26B8B928DEC35F08DEC35F05BEC37F043
:1019B0006BEC33F0200E54EC0BF0E8CF2FF5050163
:1019C0002F51FF0AD8A4ECEF0CF02F6B200E0C6EF9
:1019D0002FC50BF03DEC0BF00501010E306F3C0EF6
:1019E000316F250E54EC0BF0E8CF00F1260E54ECCD
:1019F0000BF0E8CF01F1270E54EC0BF0E8CF02F129
:101A0000280E54EC0BF0E8CF03F1010103AF23EFF4
:101A10000DF050EC30F0250E0C6E00C10BF03DECDB
:101A20000BF0260E0C6E01C10BF03DEC0BF0270EF7
:101A30000C6E02C10BF03DEC0BF0280E0C6E03C1D6
:101A40000BF03DEC0BF000C157F501C158F502C198
:101A500059F503C15AF500C15BF501C15CF502C13E
:101A60005DF503C15EF5290E54EC0BF0E8CF5FF590
:101A7000050160515F5DD8A05FC560F5210E54EC93
:101A80000BF0E8CF00F1220E54EC0BF0E8CF01F19F
:101A9000230E54EC0BF0E8CF02F1240E54EC0BF0C3
:101AA000E8CF03F1010103AF84EF0DF050EC30F00B
:101AB000210E0C6E00C10BF03DEC0BF0220E0C6EF3
:101AC00001C10BF03DEC0BF0230E0C6E02C10BF0CC
:101AD0003DEC0BF0240E0C6E03C10BF03DEC0BF053
:101AE000210E54EC0BF0E8CF00F1220E54EC0BF079
:101AF000E8CF01F1230E54EC0BF0E8CF02F1240EF5
:101B000054EC0BF0E8CF03F100C161F501C162F5BF
:101B100002C163F503C164F5B3EC32F099EC31F026
:101B2000F1EC30F037A0F5EF0DF005012F51020A6E
:101B300016E005012F51030A19E005012F51040A8F
:101B400024E005012F51050A2BE005012F51060A5B
:101B500039E005012F51070A3FE0F5EF0DF0602F46
:101B6000F2EF0DF05FC560F5F5EF0DF0B0C500F1D7
:101B700001010F0E001701010051000A36E00101BA
:101B80000051050A32E0F2EF0DF0B0C500F101019D
:101B90000F0E001701010051000A27E0F2EF0DF0CF
:101BA0000501B051000A21E00501B051150A1DE000
:101BB0000501B051300A19E00501B051450A15E0A0
:101BC000F2EF0DF00501B051000A0FE00501B05130
:101BD000300A0BE0F2EF0DF00501B051000A05E00C
:101BE000F2EF0DF081BA9AEF37F007900001F28E14
:101BF000F28C12AE03D012BC4AEF19F007B093EF8B
:101C00002CF00FB08FEF25F010BE8FEF25F012B83B
:101C10008FEF25F000011650010AD8B4B1EF1DF086
:101C200081BA1BEF0EF000011650040AD8B4F6EF8B
:101C30001BF021EF0EF000011650040AD8B4DCEFBF
:101C40001DF00301805181197F0BD8B493EF2CF064
:101C500013EE00F081517F0BE126812BE7CFE8FFE7
:101C6000E00BD8B493EF2CF023EE82F0C2513F0B7F
:101C7000D926E7CFDFFFC22BDF50780AD8A493EF35
:101C80002CF0078092C100F193C101F194C102F1DF
:101C900095C103F10101040E046F000E056F000EE3
:101CA000066F000E076F55EC2FF000AF61EF0EF0DE
:101CB0000101030E926F000E936F000E946F000EE1
:101CC000956F03018251720AD8B410EF25F082514A
:101CD000520AD8B410EF25F08251750AD8B410EF2B
:101CE00025F08251680AD8B4DFEF0EF08251630A02
:101CF000D8B44DEF29F08251690AD8B4D5EF20F05D
:101D000082517A0AD8B4E8EF21F08251490AD8B456
:101D100074EF20F08251500AD8B492EF1FF0825134
:101D2000700AD8B4D5EF1FF08251540AD8B400EF2E
:101D300020F08251740AD8B446EF20F08251410A53
:101D4000D8B4E4EF0FF082514B0AD8B4E1EF0EF0B3
:101D500082516D0AD8B454EF14F082514D0AD8B4B0
:101D60006DEF14F08251730AD8B440EF24F0825121
:101D7000530AD8B4A5EF24F082514C0AD8B4FCEF32
:101D800014F08251590AD8B4A5EF13F012AE01D065
:101D9000128C84EF29F0040114EE00F080517F0BC7
:101DA000E12682C4E7FF802B120004010D0E826F32
:101DB000CBEC0EF00A0E826FCBEC0EF0120082EF2D
:101DC00029F004014B0E826FCBEC0EF004012C0EB7
:101DD000826FCBEC0EF081B802D036B630D0030162
:101DE0008351430AD8B426EF0FF003018351630AED
:101DF000D8B428EF0FF003018351520AD8B42AEF68
:101E00000FF003018351720AD8B42CEF0FF00301D5
:101E10008351470AD8B42EEF0FF003018351670AAC
:101E2000D8B430EF0FF003018351540AD8B432EF25
:101E30000FF003018351740AD8B4A2EF0FF003012D
:101E40008351550AD8B434EF0FF083D036807BD05D
:101E5000369079D0368277D0369275D0368473D06A
:101E6000369471D036866FD084C330F185C331F19A
:101E700086C332F187C333F10101296B9EEC30F048
:101E800015EC30F000C104F101C105F102C106F109
:101E900003C107F191EC30F0200EF86EF76AF66A94
:101EA0000900F5CF2CF10900F5CF2DF10900F5CF90
:101EB0002EF10900F5CF2FF10900F5CF30F109001F
:101EC000F5CF31F10900F5CF32F10900F5CF33F14B
:101ED0000101296B9EEC30F015EC30F055EC2FF041
:101EE000010100677BEF0FF001677BEF0FF00267E6
:101EF0007BEF0FF0036701D025D004014E0E826FF7
:101F0000CBEC0EF004016F0E826FCBEC0EF00401EF
:101F10004D0E826FCBEC0EF00401610E826FCBECA4
:101F20000EF00401740E826FCBEC0EF00401630E10
:101F3000826FCBEC0EF00401680E826FCBEC0EF0DA
:101F400082EF29F03696CD0E0C6E36C00BF03DECCC
:101F50000BF0CD0E54EC0BF0E8CF36F036B006D0D7
:101F60000401630E826FCBEC0EF005D00401430E2A
:101F7000826FCBEC0EF036B206D00401720E826F87
:101F8000CBEC0EF005D00401520E826FCBEC0EF0BC
:101F900036B406D00401670E826FCBEC0EF005D08C
:101FA0000401470E826FCBEC0EF036B606D004016A
:101FB000740E826FCBEC0EF005D00401540E826FCC
:101FC000CBEC0EF082EF29F00401410E826FCBECD6
:101FD0000EF003018351310AD8B4C5EF12F00301AA
:101FE0008351320AD8B4F5EF11F003018351330A5B
:101FF000D8B47EEF11F003018351340AD8B46EEFE8
:1020000010F003018351350AD8B40EEF10F004012B
:102010003F0E826FCBEC0EF082EF29F0030184516A
:10202000300AD8B434EF10F003018451310AD8B427
:1020300037EF10F003018451650AD8B428EF10F08F
:1020400003018451640AD8B42BEF10F038EF10F07C
:1020500038902CEF10F03880FB0E0C6E38C00BF06F
:102060003DEC0BF038EF10F08B9038EF10F08B80D8
:102070000401350E826FCBEC0EF004012C0E826F42
:10208000CBEC0EF08BB04CEF10F00401300E826FF1
:10209000CBEC0EF051EF10F00401310E826FCBEC5F
:1020A0000EF004012C0E826FCBEC0EF0FB0E54EC04
:1020B0000BF0E8CF38F038A065EF10F00401640EA3
:1020C000826FCBEC0EF06AEF10F00401650E826FA8
:1020D000CBEC0EF06CEF10F082EF29F0CC0E54EC4C
:1020E0000BF0E8CF0BF004012C0E826FCBEC0EF05E
:1020F00003018451310AD8B492EF10F003018451E6
:10210000300AD8B494EF10F0030184514D0AD8B4CA
:102110009EEF10F003018451540AD8B4A5EF10F0DB
:10212000BCEF10F08A8401D08A940BAE04D00BACC3
:1021300002D00BBA21D0E00E0B1218D01F0E0B16D6
:102140008539E844E00B0B1211D0E00E0B1691EC30
:1021500030F085C332F186C333F10101296B9EEC67
:1021600030F015EC30F000511F0B0B12CC0E0C6E42
:102170000BC00BF03DEC0BF00401340E826FCBEC86
:102180000EF004012C0E826FCBEC0EF0CC0E54EC52
:102190000BF0E8CF1DF08AB406D00401300E826F38
:1021A000CBEC0EF005D00401310E826FCBEC0EF0BB
:1021B00004012C0E826FCBEC0EF01D38E840070BAB
:1021C000E8CF82F40401300E8227CBEC0EF004013C
:1021D0002C0E826FCBEC0EF050EC30F01D501F0B2C
:1021E000E8CF00F1F3EC2FF032C182F40401300E9D
:1021F0008227CBEC0EF033C182F40401300E82272B
:10220000CBEC0EF004012C0E826FCBEC0EF050ECF8
:1022100030F030C000F100AF0BD0FF0E016FFF0EA9
:10222000026FFF0E036F04012D0E826FCBEC0EF0D8
:10223000F3EC2FF031C182F40401300E8227CBEC95
:102240000EF032C182F40401300E8227CBEC0EF086
:1022500033C182F40401300E8227CBEC0EF004016E
:102260002C0E826FCBEC0EF050EC30F02FC000F152
:10227000F3EC2FF031C182F40401300E8227CBEC55
:102280000EF032C182F40401300E8227CBEC0EF046
:1022900033C182F40401300E8227CBEC0EF004012E
:1022A0002C0E826FCBEC0EF050EC30F031C000F110
:1022B00000AF0BD0FF0E016FFF0E026FFF0E036F1A
:1022C00004012D0E826FCBEC0EF0F3EC2FF031C138
:1022D00082F40401300E8227CBEC0EF032C182F47E
:1022E0000401300E8227CBEC0EF033C182F40401DE
:1022F000300E8227CBEC0EF082EF29F0CB0E54EC9F
:102300000BF0E8CF0BF004012C0E826FCBEC0EF03B
:1023100003018451450AD8B4A2EF11F0030184519E
:10232000440AD8B4A5EF11F003018451300AD8B49F
:10233000A8EF11F003018451310AD8B4ACEF11F0C9
:10234000B7EF11F00B9EB1EF11F00B8EB1EF11F062
:10235000FC0E0B16B1EF11F0FC0E0B160B80B1EF5B
:1023600011F0CB0E0C6E0BC00BF03DEC0BF004012A
:10237000330E826FCBEC0EF004012C0E826FCBEC8F
:102380000EF0CB0E54EC0BF0E8CF1CF01CBED0EFDF
:1023900011F00401450E826FCBEC0EF0D5EF11F079
:1023A0000401440E826FCBEC0EF004012C0E826F00
:1023B000CBEC0EF00401300E826FCBEC0EF004017A
:1023C0002C0E826FCBEC0EF01CB0EEEF11F004017E
:1023D000300E826FCBEC0EF0F3EF11F00401310EF2
:1023E000826FCBEC0EF082EF29F0CA0E54EC0BF0AA
:1023F000E8CF0BF004012C0E826FCBEC0EF0030142
:102400008451450AD8B431EF12F003018451440AD3
:10241000D8B434EF12F0030184514D0AD8B43DEF23
:1024200012F003018451410AD8B437EF12F00301CE
:102430008451460AD8B43AEF12F003018451560A87
:10244000D8B445EF12F003018451500AD8B450EFCC
:1024500012F003018451520AD8B453EF12F05CEF2A
:1024600012F00B9E56EF12F00B8E56EF12F00B9CF3
:1024700056EF12F00B8C56EF12F0FC0E0B1685C3C4
:10248000E8FF030B0B1256EF12F0C70E0B1685C3B5
:10249000E8FF070BE846E846E8460B1256EF12F055
:1024A0000B8456EF12F00B9456EF12F0CA0E0C6E1E
:1024B0000BC00BF03DEC0BF0CA0E54EC0BF0E8CF68
:1024C0001BF00401320E826FCBEC0EF004012C0ED7
:1024D000826FCBEC0EF01BBE75EF12F00401450EBF
:1024E000826FCBEC0EF07AEF12F00401440E826F93
:1024F000CBEC0EF004012C0E826FCBEC0EF01BC067
:10250000E8FF030BE8CF82F40401300E8227CBEC06
:102510000EF004012C0E826FCBEC0EF01BBC98EF7A
:1025200012F00401410E826FCBEC0EF09DEF12F021
:102530000401460E826FCBEC0EF004012C0E826F6C
:10254000CBEC0EF01BC0E8FF380BE842E842E84253
:10255000E8CF82F40401300E8227CBEC0EF00401A8
:102560002C0E826FCBEC0EF01BB4BEEF12F0040108
:10257000520E826FCBEC0EF0C3EF12F00401500E3E
:10258000826FCBEC0EF082EF29F0C90E54EC0BF009
:10259000E8CF0BF004012C0E826FCBEC0EF00301A0
:1025A0008451450AD8B4E3EF12F003018451440A80
:1025B000D8B4E6EF12F0030184514D0AD8B4E9EF24
:1025C00012F0F7EF12F00B9EF1EF12F00B8EF1EF1D
:1025D00012F0F80E0B1685C3E8FF070B0B12F1EF94
:1025E00012F0C90E0C6E0BC00BF03DEC0BF00401A9
:1025F000310E826FCBEC0EF004012C0E826FCBEC0F
:102600000EF0C90E54EC0BF0E8CF1AF01ABE06D04B
:102610000401450E826FCBEC0EF005D00401440E90
:10262000826FCBEC0EF004012C0E826FCBEC0EF01F
:102630001AC0E8FF070BE8CF82F40401300E8227AE
:10264000CBEC0EF004012C0E826FCBEC0EF0078069
:1026500050EC30F02BC0E8FF003B00430043030B7D
:10266000F3EC2FF033C182F40401300E8227CBEC5F
:102670000EF004012C0E826FCBEC0EF050EC30F01B
:102680002BC001F1019F019D2CC000F10101F3EC71
:102690002FF02FC182F40401300E8227CBEC0EF014
:1026A00030C182F40401300E8227CBEC0EF031C130
:1026B00082F40401300E8227CBEC0EF032C182F49A
:1026C0000401300E8227CBEC0EF033C182F40401FA
:1026D000300E8227CBEC0EF004012C0E826FCBEC77
:1026E0000EF050EC30F02DC001F12EC000F1D8906A
:1026F00001330033D890013300330101F3EC2FF0A4
:102700002FC182F40401300E8227CBEC0EF030C1D1
:1027100082F40401300E8227CBEC0EF031C182F43A
:102720000401300E8227CBEC0EF032C182F404019A
:10273000300E8227CBEC0EF033C182F40401300E50
:102740008227CBEC0EF082EF29F0FC0E54EC0BF05C
:10275000E8CF0BF003018351520AD8B4DCEF13F039
:1027600003018351720AD8B4DFEF13F003018351E0
:10277000500AD8B4E2EF13F003018351700AD8B4C1
:10278000E5EF13F003018351550AD8B4E8EF13F0D5
:1027900003018351750AD8B4EBEF13F003018351A1
:1027A000430AD8B4F4EF13F003018351630AD8B499
:1027B000F7EF13F000EF14F00B90FAEF13F00B802B
:1027C000FAEF13F00B92FAEF13F00B82FAEF13F01B
:1027D0000B94FAEF13F00B84FAEF13F00B96FAEF69
:1027E00013F00B86FAEF13F00B98FAEF13F00B8847
:1027F000FAEF13F0FC0E0C6E0BC00BF03DEC0BF07F
:102800000401590E826FCBEC0EF0119011921194CD
:102810001198FC0E54EC0BF0E8CF0BF00BA01180DC
:102820000BA211820BA411840BA8118811A020EF18
:1028300014F00401520E826FCBEC0EF025EF14F071
:102840000401720E826FCBEC0EF011A82FEF14F082
:102850000401430E826FCBEC0EF034EF14F0040150
:10286000630E826FCBEC0EF011A23EEF14F0040168
:10287000500E826FCBEC0EF043EF14F00401700E9B
:10288000826FCBEC0EF011A44DEF14F00401550E45
:10289000826FCBEC0EF052EF14F00401750E826FD4
:1028A000CBEC0EF082EF29F004016D0E826FCBECC1
:1028B0000EF003018351300AD8B4ACEF14F00301D9
:1028C0008351310AD8B4BFEF14F003018351320AA7
:1028D000D8B4D2EF14F084EF29F004014D0E826FCA
:1028E000CBEC0EF091EC30F084C331F185C332F1C2
:1028F00086C333F10101296B9EEC30F015EC30F00A
:1029000003018351300AD8B494EF14F003018351CA
:10291000310AD8B49CEF14F003018351320AD8B4C1
:10292000A4EF14F084EF29F0FD0E0C6E00C10BF043
:102930003DEC0BF0ACEF14F0FE0E0C6E00C10BF092
:102940003DEC0BF0BFEF14F0FF0E0C6E00C10BF06E
:102950003DEC0BF0D2EF14F00401300E826FCBECA3
:102960000EF004012C0E826FCBEC0EF050EC30F028
:10297000FD0E54EC0BF0E8CF00F1E3EF14F004018E
:10298000310E826FCBEC0EF004012C0E826FCBEC7B
:102990000EF050EC30F0FE0E54EC0BF0E8CF00F1EE
:1029A000E3EF14F00401320E826FCBEC0EF050EC2A
:1029B00030F004012C0E826FCBEC0EF0FF0E54ECC5
:1029C0000BF0E8CF00F1F3EC2FF031C182F40401F9
:1029D000300E8227CBEC0EF032C182F40401300EAF
:1029E0008227CBEC0EF033C182F40401300E822733
:1029F000CBEC0EF082EF29F003018351300AD8B4FA
:102A0000F7EF19F003018351310AD8B424EF1BF01A
:102A100003018351320AD8B492EF1BF003018351B2
:102A2000330AD8B4A2EF1BF003018351340AD8B49F
:102A3000FDEF1BF003018351350AD8B4E3EF1DF01D
:102A400003018351360AD8B411EF1EF003018351FC
:102A5000370AD8B4CFEF17F003018351380AD8B43E
:102A60006DEF18F003018351460AD8B40AEF1DF048
:102A7000030183514D0AD8B448EF16F00301835186
:102A80006D0AD8B462EF16F0030183515A0AD8B424
:102A90009EEF1AF003018351490AD8B411EF1FF0D9
:102AA00003018351500AD8B443EF1EF00301835150
:102AB000540AD8B4BCEF1EF003018351630AD8B4A2
:102AC00082EF16F003018351430AD8B47AEF17F06E
:102AD00003018351730AD8B480EF16F003018351C8
:102AE000610AD8B495EF15F003018351650AD8B493
:102AF00047EF1AF003018351450AD8B455EF1AF095
:102B000003018351620AD8B463EF1AF003018351C1
:102B1000420AD8B471EF1AF003018351760AD8B48F
:102B20007FEF1AF0D8A484EF29F004014C0E826FD5
:102B3000CBEC0EF00401610E826FCBEC0EF099EC41
:102B400031F004012C0E826FCBEC0EF050EC30F023
:102B5000AFC500F10101F3EC2FF031C182F40401A3
:102B6000300E8227CBEC0EF032C182F40401300E1D
:102B70008227CBEC0EF033C182F40401300E8227A1
:102B8000CBEC0EF004012C0E826FCBEC0EF050EC6F
:102B900030F0B0C500F10101F3EC2FF031C182F447
:102BA0000401300E8227CBEC0EF032C182F4040116
:102BB000300E8227CBEC0EF033C182F40401300ECC
:102BC0008227CBEC0EF004012C0E826FCBEC0EF0C2
:102BD00050EC30F0B1C500F10101F3EC2FF031C140
:102BE00082F40401300E8227CBEC0EF032C182F465
:102BF0000401300E8227CBEC0EF033C182F40401C5
:102C0000300E8227CBEC0EF004012C0E826FCBEC41
:102C10000EF050EC30F0B2C500F10101F3EC2FF0F2
:102C200031C182F40401300E8227CBEC0EF032C1A8
:102C300082F40401300E8227CBEC0EF033C182F413
:102C40000401300E8227CBEC0EF004012C0E826FB3
:102C5000CBEC0EF050EC30F0B6C500F10101F3EC16
:102C60002FF031C182F40401300E8227CBEC0EF03C
:102C700032C182F40401300E8227CBEC0EF033C156
:102C800082F40401300E8227CBEC0EF03FEF1EF0F1
:102C900091EC30F084C333F19EEC30F015EC30F061
:102CA000200E0C6E00C10BF03DEC0BF000C12FF5B7
:102CB00005012F51000A06E005012F51010A02E02B
:102CC00033EC32F004014C0E826FCBEC0EF00401B9
:102CD0004D0E826FCBEC0EF004012C0E826FCBEC0C
:102CE0000EF050EC30F02FC500F1F3EC2FF033C1B3
:102CF00082F40401300E8227CBEC0EF03FEF1EF081
:102D00009AEF37F004014C0E826FCBEC0EF0040109
:102D1000630E826FCBEC0EF0F1EC30F004012C0E60
:102D2000826FCBEC0EF097EC16F03FEF1EF050ECFC
:102D300030F0B5C500F10101003B0F0E0017F3ECB8
:102D40002FF033C182F40401300E8227CBEC0EF059
:102D5000B5C500F101010F0E01010017F3EC2FF0D2
:102D600033C182F40401300E8227CBEC0EF0040153
:102D70002D0E826FCBEC0EF0B4C500F10101003BCB
:102D80000F0E0017F3EC2FF033C182F40401300E64
:102D90008227CBEC0EF0B4C500F101010F0E01014A
:102DA0000017F3EC2FF033C182F40401300E8227B8
:102DB000CBEC0EF004012D0E826FCBEC0EF0B3C500
:102DC00000F10101003B0F0E0017F3EC2FF033C1AF
:102DD00082F40401300E8227CBEC0EF0B3C500F173
:102DE00001010F0E01010017F3EC2FF033C182F443
:102DF0000401300E8227CBEC0EF00401200E826F0E
:102E0000CBEC0EF0B2C500F10F0E01010017F3EC90
:102E10002FF033C182F40401300E8227CBEC0EF088
:102E20000401200E826FCBEC0EF0B1C500F1010160
:102E30000101003B0F0E0017F3EC2FF033C182F4B9
:102E40000401300E8227CBEC0EF0B1C500F1010178
:102E50000F0E01010017F3EC2FF033C182F40401CF
:102E6000300E8227CBEC0EF004013A0E826FCBECD1
:102E70000EF0B0C500F10101003B0F0E0017F3EC9E
:102E80002FF033C182F40401300E8227CBEC0EF018
:102E9000B0C500F101010F0E01010017F3EC2FF096
:102EA00033C182F40401300E8227CBEC0EF0040112
:102EB0003A0E826FCBEC0EF0AFC500F10101003B82
:102EC0000F0E0017F3EC2FF033C182F40401300E23
:102ED0008227CBEC0EF0AFC500F101010F0E0017F9
:102EE000F3EC2FF033C182F40401300E8227CBECD7
:102EF0000EF0120084C3E8FF0F0BE83AE8CFB5F5F7
:102F000085C3E8FF0F0B0501B51387C3E8FF0F0B5F
:102F1000E83AE8CFB4F588C3E8FF0F0B0501B41316
:102F20008AC3E8FF0F0BE83AE8CFB3F58BC3E8FF9D
:102F30000F0B0501B3138DC3E8FF0F0BE8CFB2F5FC
:102F40008FC3E8FF0F0BE83AE8CFB1F590C3E8FF75
:102F50000F0B0501B11392C3E8FF0F0BE83AE8CF5E
:102F6000B0F593C3E8FF0F0B0501B01395C3E8FF5D
:102F70000F0BE83AE8CFAFF596C3E8FF0F0B05015A
:102F8000AF134CEC31F004014C0E826FCBEC0EF021
:102F90000401430E826FCBEC0EF08CEF16F0078429
:102FA00004014C0E826FCBEC0EF00401370E826FE1
:102FB000CBEC0EF004012C0E826FCBEC0EF0050171
:102FC0002E51130A06E005012E51170A0DE06AEF93
:102FD00018F00101000E006F000E016F100E026F5D
:102FE000000E036FFDEF17F00101000E006F000EE1
:102FF000016F000E026F010E036FF3EC2FF02AC178
:1030000082F40401300E8227CBEC0EF02BC182F447
:103010000401300E8227CBEC0EF02CC182F40401A7
:10302000300E8227CBEC0EF02DC182F40401300E5D
:103030008227CBEC0EF02EC182F40401300E8227E1
:10304000CBEC0EF02FC182F40401300E8227CBECC2
:103050000EF030C182F40401300E8227CBEC0EF06A
:1030600031C182F40401300E8227CBEC0EF032C164
:1030700082F40401300E8227CBEC0EF033C182F4CF
:103080000401300E8227CBEC0EF004012C0E826F6F
:10309000CBEC0EF00101100E006F000E016F000E60
:1030A000026F000E036FF3EC2FF031C182F40401C4
:1030B000300E8227CBEC0EF032C182F40401300EC8
:1030C0008227CBEC0EF033C182F40401300E82274C
:1030D000CBEC0EF007943FEF1EF00501216B226B45
:1030E000236B246B04014C0E826FCBEC0EF00401B9
:1030F000380E826FCBEC0EF004012C0E826FCBECFD
:103100000EF00101100E006F000E016F000E026F35
:10311000000E036FF3EC2FF02AC182F40401300E8D
:103120008227CBEC0EF02BC182F40401300E8227F3
:10313000CBEC0EF02CC182F40401300E8227CBECD4
:103140000EF02DC182F40401300E8227CBEC0EF07C
:103150002EC182F40401300E8227CBEC0EF02FC179
:1031600082F40401300E8227CBEC0EF030C182F4E1
:103170000401300E8227CBEC0EF031C182F4040141
:10318000300E8227CBEC0EF032C182F40401300EF7
:103190008227CBEC0EF033C182F40401300E82277B
:1031A000CBEC0EF004012C0E826FCBEC0EF025C59B
:1031B00000F126C501F127C502F128C503F101017F
:1031C000100E046F000E056F000E066F000E076FE5
:1031D00086EC2FF000C133F501C134F502C135F59D
:1031E00003C136F5F3EC2FF02AC182F40401300E4E
:1031F0008227CBEC0EF02BC182F40401300E822723
:10320000CBEC0EF02CC182F40401300E8227CBEC03
:103210000EF02DC182F40401300E8227CBEC0EF0AB
:103220002EC182F40401300E8227CBEC0EF02FC1A8
:1032300082F40401300E8227CBEC0EF030C182F410
:103240000401300E8227CBEC0EF031C182F4040170
:10325000300E8227CBEC0EF032C182F40401300E26
:103260008227CBEC0EF033C182F40401300E8227AA
:10327000CBEC0EF0D5EC0EF00501336747EF19F0FB
:10328000346747EF19F0356747EF19F0366702D01A
:10329000E6EF19F0129E129C21C500F122C501F142
:1032A00023C502F124C503F1899A400EC76E200E92
:1032B000C66E9E96C69E0B0EC96EFF0E9EB602D0BF
:1032C000E82EFCD79E96C69E02C1C9FFFF0E9EB691
:1032D00002D0E82EFCD79E96C69E01C1C9FFFF0E04
:1032E0009EB602D0E82EFCD79E96C69E00C1C9FFAE
:1032F000FF0E9EB602D0E82EFCD79E96C69EC952FF
:10330000FF0E9EB602D0E82EFCD70501100E326FDC
:10331000040114EE00F080517F0BE1269E96C69EBC
:10332000C952FF0E9EB602D0E82EFCD7C9CFE7FFE8
:103330000401802B0501322F88EF19F0898A33C5EB
:1033400000F134C501F135C502F136C503F10101C3
:10335000010E046F000E056F000E066F000E076F62
:1033600055EC2FF000C133F501C134F502C135F53C
:1033700003C136F505013367C5EF19F03467C5EFB2
:1033800019F03567C5EF19F0366702D0E6EF19F08E
:1033900021C500F122C501F123C502F124C503F1C5
:1033A0000101100E046F000E056F000E066F000E77
:1033B000076F5AEC2FF000C121F501C122F502C1BF
:1033C00023F503C124F5128E84EF29F00401450E84
:1033D000826FCBEC0EF004014F0E826FCBEC0EF03F
:1033E0000401460E826FCBEC0EF03FEF1EF0078417
:1033F0005BEC37F050EC30F02DC500F1F3EC2FF022
:1034000004014C0E826FCBEC0EF00401300E826F83
:10341000CBEC0EF004012C0E826FCBEC0EF031C120
:1034200082F40401300E8227CBEC0EF032C182F41C
:103430000401300E8227CBEC0EF033C182F404017C
:10344000300E8227CBEC0EF004012C0E826FCBECF9
:103450000EF050EC30F02EC500F1F3EC2FF031C13E
:1034600082F40401300E8227CBEC0EF032C182F4DC
:103470000401300E8227CBEC0EF033C182F404013C
:10348000300E8227CBEC0EF007943FEF1EF00401C4
:103490004C0E826FCBEC0EF00401650E826FCBEC0C
:1034A0000EF00FEC33F03FEF1EF004014C0E826F74
:1034B000CBEC0EF00401450E826FCBEC0EF026EC47
:1034C00033F03FEF1EF004014C0E826FCBEC0EF098
:1034D0000401620E826FCBEC0EF054EC33F03FEF40
:1034E0001EF004014C0E826FCBEC0EF00401420E74
:1034F000826FCBEC0EF03DEC33F03FEF1EF0040199
:103500004C0E826FCBEC0EF00401760E826FCBEC8A
:103510000EF004012C0E826FCBEC0EF010A807D039
:103520000401310E826FCBEC0EF03FEF1EF0040170
:10353000300E826FCBEC0EF03FEF1EF004014C0E0C
:10354000826FCBEC0EF004015A0E826FCBEC0EF0C2
:1035500004012C0E826FCBEC0EF05BEC37F050ECDC
:1035600030F005012E51130A06E005012E51170A0D
:103570000DE0CFEF1AF00101000E006F000E016F99
:10358000100E026F000E036FCFEF1AF00101000E54
:10359000006F000E016F000E026F010E036F01013C
:1035A000100E046F000E056F000E066F000E076F01
:1035B00086EC2FF0F3EC2FF02AC182F40401300ED8
:1035C0008227CBEC0EF02BC182F40401300E82274F
:1035D000CBEC0EF02CC182F40401300E8227CBEC30
:1035E0000EF02DC182F40401300E8227CBEC0EF0D8
:1035F0002EC182F40401300E8227CBEC0EF02FC1D5
:1036000082F40401300E8227CBEC0EF030C182F43C
:103610000401300E8227CBEC0EF031C182F404019C
:10362000300E8227CBEC0EF032C182F40401300E52
:103630008227CBEC0EF033C182F40401300E8227D6
:10364000CBEC0EF03FEF1EF0078404014C0E826FAE
:10365000CBEC0EF00401310E826FCBEC0EF00401C6
:103660002C0E826FCBEC0EF025C500F126C501F1C2
:1036700027C502F128C503F10101100E046F000EE9
:10368000056F000E066F000E076F86EC2FF0F3EC4F
:103690002FF02AC182F40401300E8227CBEC0EF009
:1036A0002BC182F40401300E8227CBEC0EF02CC12A
:1036B00082F40401300E8227CBEC0EF02DC182F48F
:1036C0000401300E8227CBEC0EF02EC182F40401EF
:1036D000300E8227CBEC0EF02FC182F40401300EA5
:1036E0008227CBEC0EF030C182F40401300E822729
:1036F000CBEC0EF031C182F40401300E8227CBEC0A
:103700000EF032C182F40401300E8227CBEC0EF0B1
:1037100033C182F40401300E8227CBEC0EF0079403
:103720003FEF1EF0078404014C0E826FCBEC0EF0CD
:103730000401320E826FCBEC0EF043EC35F00794AF
:103740003FEF1EF0078438B0A8EF1BF0BBEF1BF073
:10375000010E166E04014C0E826FCBEC0EF00401CC
:10376000330E826FCBEC0EF0A0EC35F0000E166E2F
:1037700007942FEF1BF0020E166EA0EC35F08B8035
:103780000501010E306F3C0E316F01015E6B5F6B06
:10379000606B616B626B636B646B656B666B676BB5
:1037A000686B696B536B546BCF6ACE6A0F9A0F9C30
:1037B0000F9E030E166E04014C0E826FCBEC0EF0C2
:1037C0000401330E826FCBEC0EF004012C0E826FDD
:1037D000CBEC0EF004012D0E826FCBEC0EF0040149
:1037E000310E826FCBEC0EF082EF29F0A0EC35F0B9
:1037F000000E166E8B9084EF29F0078404014C0EA6
:10380000826FCBEC0EF00401340E826FCBEC0EF025
:1038100004012C0E826FCBEC0EF091EC30F084C3DF
:103820002AF185C32BF186C32CF187C32DF188C300
:103830002EF189C32FF18AC330F18BC331F18CC3D0
:1038400032F18DC333F10101296B9EEC30F015ECA0
:1038500030F0100E046F000E056F000E066F000EA4
:10386000076F66EC2FF000C121F501C122F502C1FE
:1038700023F503C124F50EEC37F038C5AFF539C593
:10388000B0F53AC5B1F53BC5B2F53CC5B3F53DC59C
:10389000B4F53EC5B5F597EC16F004012C0E826F19
:1038A000CBEC0EF03FC500F140C501F141C502F17E
:1038B00042C503F10101000E046F000E056F010EF9
:1038C000066F000E076F86EC2FF0F3EC2FF02967E0
:1038D0006CEF1CF071EF1CF004012D0E826FCBEC2D
:1038E0000EF030C182F40401300E8227CBEC0EF0D2
:1038F00031C182F40401300E8227CBEC0EF00401BA
:103900002E0E826FCBEC0EF032C182F40401300E29
:103910008227CBEC0EF033C182F40401300E8227F3
:10392000CBEC0EF004012C0E826FCBEC0EF050ECC1
:1039300030F043C500F144C501F1AEEC2AF00401BA
:103940002C0E826FCBEC0EF050EC30F045C500F140
:10395000F3EC2FF031C182F40401300E8227CBEC5E
:103960000EF032C182F40401300E8227CBEC0EF04F
:1039700033C182F40401300E8227CBEC0EF0040137
:103980002C0E826FCBEC0EF037C5E8FFE8B806D0FE
:103990000401300E826FCBEC0EF005D00401310E25
:1039A000826FCBEC0EF004012C0E826FCBEC0EF08C
:1039B00037C5E8FFE8BA06D00401300E826FCBECC1
:1039C0000EF025D00401310E826FCBEC0EF0040115
:1039D0002C0E826FCBEC0EF050EC30F046C500F1AF
:1039E000F3EC2FF031C182F40401300E8227CBECCE
:1039F0000EF032C182F40401300E8227CBEC0EF0BF
:103A000033C182F40401300E8227CBEC0EF0079410
:103A10003FEF1EF091EC30F085C32AF186C32BF105
:103A200087C32CF188C32DF189C32EF18AC32FF1EE
:103A30008BC330F18CC331F18DC332F18EC333F1BE
:103A40000101296B9EEC30F015EC30F00101010E04
:103A5000046F000E056F000E066F000E076F55EC29
:103A60002FF0100E046F000E056F000E066F000E93
:103A7000076F66EC2FF000C129F501C12AF502C1DC
:103A80002BF503C12CF5CAEC34F004014C0E826F07
:103A9000CBEC0EF00401460E826FCBEC0EF004016D
:103AA0002C0E826FCBEC0EF025C500F126C501F17E
:103AB00027C502F128C503F10101100E046F000EA5
:103AC000056F000E066F000E076F86EC2FF0F3EC0B
:103AD0002FF02AC182F40401300E8227CBEC0EF0C5
:103AE0002BC182F40401300E8227CBEC0EF02CC1E6
:103AF00082F40401300E8227CBEC0EF02DC182F44B
:103B00000401300E8227CBEC0EF02EC182F40401AA
:103B1000300E8227CBEC0EF02FC182F40401300E60
:103B20008227CBEC0EF030C182F40401300E8227E4
:103B3000CBEC0EF031C182F40401300E8227CBECC5
:103B40000EF032C182F40401300E8227CBEC0EF06D
:103B500033C182F40401300E8227CBEC0EF03FEF2C
:103B60001EF038B0B6EF1DF0020E166EA0EC35F068
:103B700000011650020AD8B4C3EF1DF0050E166EF0
:103B800037809AEF37F08B8001015E6B5F6B606B63
:103B9000616B626B636B646B656B666B676B686BA9
:103BA000696B536B546BCF6ACE6A0F9A0F9C0F9E52
:103BB000030E166E84EF29F0A0EC35F0050E166E9C
:103BC00037809AEF37F004014C0E826FCBEC0EF089
:103BD0000401350E826FCBEC0EF004012C0E826FC7
:103BE000CBEC0EF050EC30F00784B9C500F107942F
:103BF000F3EC2FF031C182F40401300E8227CBECBC
:103C00000EF032C182F40401300E8227CBEC0EF0AC
:103C100033C182F40401300E8227CBEC0EF03FEF6B
:103C20001EF063EC35F050EC30F037C500F1F3ECEA
:103C30002FF004014C0E826FCBEC0EF00401360E17
:103C4000826FCBEC0EF004012C0E826FCBEC0EF0E9
:103C500031C182F40401300E8227CBEC0EF032C168
:103C600082F40401300E8227CBEC0EF033C182F4D3
:103C70000401300E8227CBEC0EF03FEF1EF0D5ECA6
:103C80000EF084EF29F004014C0E826FCBEC0EF0A5
:103C90000401500E826FCBEC0EF004012C0E826FEB
:103CA000CBEC0EF085C32AF186C32BF187C32CF130
:103CB00088C32DF189C32EF18AC32FF18BC330F154
:103CC0008CC331F18DC332F18EC333F101019EEC0F
:103CD00030F015EC30F003018451530A0DE003017C
:103CE00084514D0A38E00401780E826FCBEC0EF05F
:103CF000D5EC0EF084EF29F00401530E826FCBEC6B
:103D00000EF0250E0C6E00C10BF03DEC0BF0260EF4
:103D10000C6E01C10BF03DEC0BF0270E0C6E02C1D6
:103D20000BF03DEC0BF0280E0C6E03C10BF03DECDC
:103D30000BF000C157F501C158F502C159F503C197
:103D40005AF500C15BF501C15CF502C15DF503C127
:103D50005EF520EF1FF004014D0E826FCBEC0EF0EC
:103D6000290E0C6E00C10BF03DEC0BF000C15FF5AD
:103D700000C160F520EF1FF004014C0E826FCBEC08
:103D80000EF00401540E826FCBEC0EF004012C0EE9
:103D9000826FCBEC0EF084C32AF185C32BF186C36E
:103DA0002CF187C32DF188C32EF189C32FF18AC36B
:103DB00030F18BC331F18DC332F18EC333F1010188
:103DC0009EEC30F015EC30F00101000E046F000E97
:103DD000056F010E066F000E076F66EC2FF0210EC7
:103DE0000C6E00C10BF03DEC0BF0220E0C6E01C10D
:103DF0000BF03DEC0BF0230E0C6E02C10BF03DEC12
:103E00000BF0240E0C6E03C10BF03DEC0BF000C167
:103E100061F501C162F502C163F503C164F520EFEC
:103E20001FF004014C0E826FCBEC0EF00401490E22
:103E3000826FCBEC0EF004012C0E826FCBEC0EF0F7
:103E4000250E54EC0BF0E8CF00F1260E54EC0BF0ED
:103E5000E8CF01F1270E54EC0BF0E8CF02F1280E69
:103E600054EC0BF0E8CF03F1F3EC2FF0B6EC2DF0AF
:103E70000401730E826FCBEC0EF004012C0E826FE6
:103E8000CBEC0EF050EC30F0290E54EC0BF0E8CFF8
:103E900000F1F3EC2FF0B6EC2DF004016D0E826F03
:103EA000CBEC0EF004012C0E826FCBEC0EF05BC558
:103EB00000F15CC501F15DC502F15EC503F1F3ECF3
:103EC0002FF0B6EC2DF00401730E826FCBEC0EF0E8
:103ED00004012C0E826FCBEC0EF050EC30F060C57C
:103EE00000F1F3EC2FF0B6EC2DF004016D0E826FB3
:103EF000CBEC0EF004012C0E826FCBEC0EF061C502
:103F000000F162C501F163C502F164C503F19FECE4
:103F100029F004012C0E826FCBEC0EF0D5EC0EF0E4
:103F200084EF29F083C32AF184C32BF185C32CF1DC
:103F300086C32DF187C32EF188C32FF189C330F1D9
:103F40008AC331F18BC332F18CC333F101019EEC92
:103F500030F015EC30F0160E0C6E00C10BF03DEC9D
:103F60000BF0170E0C6E01C10BF03DEC0BF0180EB0
:103F70000C6E02C10BF03DEC0BF0190E0C6E03C180
:103F80000BF03DEC0BF000C18EF101C18FF102C1CD
:103F900090F103C191F100C192F101C193F102C10D
:103FA00094F103C195F174EF20F083C32AF184C327
:103FB0002BF185C32CF186C32DF187C32EF188C365
:103FC0002FF189C330F18AC331F18BC332F18CC335
:103FD00033F101019EEC30F015EC30F000C18EF1B0
:103FE00001C18FF102C190F103C191F100C192F1C1
:103FF00001C193F102C194F103C195F174EF20F076
:1040000083C32AF184C32BF185C32CF186C32DF120
:1040100087C32EF188C32FF189C330F18AC331F1F0
:104020008CC332F18DC333F101019EEC30F015ECFD
:1040300030F00101000E046F000E056F010E066FD7
:10404000000E076F66EC2FF01A0E0C6E00C10BF01D
:104050003DEC0BF01B0E0C6E01C10BF03DEC0BF0B8
:104060001C0E0C6E02C10BF03DEC0BF01D0E0C6E25
:1040700003C10BF03DEC0BF000C196F101C197F1CB
:1040800002C198F103C199F174EF20F083C32AF1C2
:1040900084C32BF185C32CF186C32DF187C32EF188
:1040A00088C32FF189C330F18AC331F18CC332F157
:1040B0008DC333F101019EEC30F015EC30F00101BD
:1040C000000E046F000E056F010E066F000E076FE5
:1040D00066EC2FF000C196F101C197F102C198F191
:1040E00003C199F174EF20F0160E54EC0BF0E8CFF9
:1040F00000F1170E54EC0BF0E8CF01F1180E54EC60
:104100000BF0E8CF02F1190E54EC0BF0E8CF03F1FD
:10411000F3EC2FF0B6EC2DF00401730E826FCBECB4
:104120000EF004012C0E826FCBEC0EF08EC100F16C
:104130008FC101F190C102F191C103F1F3EC2FF0B5
:10414000B6EC2DF00401730E826FCBEC0EF004017F
:104150002C0E826FCBEC0EF01A0E54EC0BF0E8CF65
:1041600000F11B0E54EC0BF0E8CF01F11C0E54ECE7
:104170000BF0E8CF02F11D0E54EC0BF0E8CF03F189
:104180009FEC29F004012C0E826FCBEC0EF096C14F
:1041900000F197C101F198C102F199C103F19FECBF
:1041A00029F0D5EC0EF084EF29F00401690E826F3E
:1041B000CBEC0EF004012C0E826FCBEC0EF0010163
:1041C000040E006F000E016F000E026F000E036FF1
:1041D000F3EC2FF02CC182F40401300E8227CBECDB
:1041E0000EF02DC182F40401300E8227CBEC0EF0CC
:1041F0002EC182F40401300E8227CBEC0EF02FC1C9
:1042000082F40401300E8227CBEC0EF030C182F430
:104210000401300E8227CBEC0EF031C182F4040190
:10422000300E8227CBEC0EF032C182F40401300E46
:104230008227CBEC0EF033C182F40401300E8227CA
:10424000CBEC0EF004012C0E826FCBEC0EF00101D2
:10425000060E006F000E016F000E026F000E036F5E
:10426000F3EC2FF02CC182F40401300E8227CBEC4A
:104270000EF02DC182F40401300E8227CBEC0EF03B
:104280002EC182F40401300E8227CBEC0EF02FC138
:1042900082F40401300E8227CBEC0EF030C182F4A0
:1042A0000401300E8227CBEC0EF031C182F4040100
:1042B000300E8227CBEC0EF032C182F40401300EB6
:1042C0008227CBEC0EF033C182F40401300E82273A
:1042D000CBEC0EF004012C0E826FCBEC0EF0010142
:1042E0003F0E006F000E016F000E026F000E036F95
:1042F000F3EC2FF02CC182F40401300E8227CBECBA
:104300000EF02DC182F40401300E8227CBEC0EF0AA
:104310002EC182F40401300E8227CBEC0EF02FC1A7
:1043200082F40401300E8227CBEC0EF030C182F40F
:104330000401300E8227CBEC0EF031C182F404016F
:10434000300E8227CBEC0EF032C182F40401300E25
:104350008227CBEC0EF033C182F40401300E8227A9
:10436000CBEC0EF004012C0E826FCBEC0EF0200E85
:10437000F86EF76AF66A04010900F5CF82F4CBEC17
:104380000EF00900F5CF82F4CBEC0EF00900F5CF6A
:1043900082F4CBEC0EF00900F5CF82F4CBEC0EF0FA
:1043A0000900F5CF82F4CBEC0EF00900F5CF82F4D2
:1043B000CBEC0EF00900F5CF82F4CBEC0EF0090047
:1043C000F5CF82F4CBEC0EF0D5EC0EF084EF29F0B3
:1043D0008351630AD8A482EF29F08451610AD8A4DA
:1043E00082EF29F085516C0AD8A482EF29F086511A
:1043F000410A3FE08651440A1BE08651420AD8B484
:104400004CEF22F08651350AD8B40EEF2BF08651CE
:10441000360AD8B463EF2BF08651370AD8B4CCEF04
:104420002BF08651380AD8B42AEF2CF082EF29F00D
:104430000798079A04017A0E826FCBEC0EF0040104
:10444000780E826FCBEC0EF00401640E826FCBEC21
:104450000EF00401550E826FCBEC0EF035EF22F01A
:1044600004014C0E826FCBEC0EF0D5EC0EF084EF15
:1044700029F00788079A04017A0E826FCBEC0EF0C0
:104480000401410E826FCBEC0EF00401610E826FCD
:10449000CBEC0EF029EF22F00798078A04017A0E80
:1044A000826FCBEC0EF00401420E826FCBEC0EF06B
:1044B0000401610E826FCBEC0EF029EF22F00101B6
:1044C00066676AEF22F067676AEF22F068676AEF53
:1044D00022F0696716D001014F6776EF22F050672E
:1044E00076EF22F0516776EF22F052670AD0010191
:1044F000000E006F000E016F000E026F000E036FC2
:10450000120011B80AD00101620E046F010E056F8E
:10451000000E066F000E076F09D00101A70E046F91
:10452000020E056F000E066F000E076F66C100F1E8
:1045300067C101F168C102F169C103F155EC2FF0C7
:1045400003BF13EF23F0119A119C0101000E046FB9
:10455000A80E056F550E066F020E076F66C100F1BB
:1045600067C101F168C102F169C103F166C18AF155
:1045700067C18BF168C18CF169C18DF155EC2FF0E9
:1045800003BF0BD00101000E8A6FA80E8B6F550E72
:104590008C6F020E8D6F118A119C0E0E54EC0BF075
:1045A000E8CF18F10F0E54EC0BF0E8CF19F1100E14
:1045B00054EC0BF0E8CF1AF1110E54EC0BF0E8CFED
:1045C0001BF19EEC2EF08AC104F18BC105F18CC168
:1045D00006F18DC107F155EC2FF0078262EC2EF049
:1045E0009EEC2EF0079262EC2EF08AC100F18BC196
:1045F00001F18CC102F18DC103F1079262EC2EF042
:10460000CC0E046FE00E056F870E066F050E076F68
:1046100055EC2FF000C118F101C119F102C11AF1D6
:1046200003C11BF140D013AA18EF23F0138E139A85
:10463000119C119A0101800E006F1A0E016F060E77
:10464000026F000E036F4FC104F150C105F151C15B
:1046500006F152C107F155EC2FF003AF05D050EC35
:1046600030F0118C119A12000E0E54EC0BF0E8CFC2
:1046700018F10F0E54EC0BF0E8CF19F1100E54ECBA
:104680000BF0E8CF1AF1110E54EC0BF0E8CF1BF150
:104690004FC100F150C101F151C102F152C103F10A
:1046A000078262EC2EF018C100F119C101F11AC1A4
:1046B00002F11BC103F112000784BAC166F1BBC14C
:1046C00067F1BCC168F1BDC169F14BC14FF14CC18B
:1046D00050F14DC151F14EC152F157C159F158C17C
:1046E0005AF10794010166677DEF23F067677DEF5C
:1046F00023F068677DEF23F0696716D001014F67EB
:1047000089EF23F0506789EF23F0516789EF23F099
:1047100052670AD00101000E006F000E016F000EFB
:10472000026F000E036F120011B80AD00101620E71
:10473000046F010E056F000E066F000E076F09D0A3
:104740000101A70E046F020E056F000E066F000E2A
:10475000076F66C100F167C101F168C102F169C16B
:1047600003F155EC2FF003BF15EF24F00101000E0B
:10477000046FA80E056F550E066F020E076F66C117
:1047800000F167C101F168C102F169C103F166C1BD
:104790008AF167C18BF168C18CF169C18DF155EC6B
:1047A0002FF003BF09D00101000E8A6FA80E8B6F96
:1047B000550E8C6F020E8D6F9EEC2EF000C104F131
:1047C00001C105F102C106F103C107F1000E006F3E
:1047D000A00E016F980E026F7B0E036F86EC2FF018
:1047E00000C118F101C119F102C11AF103C11BF195
:1047F000000E006FA00E016F980E026F7B0E036F0C
:104800008AC104F18BC105F18CC106F18DC107F19C
:1048100086EC2FF018C104F119C105F11AC106F197
:104820001BC107F155EC2FF012000101A80E006F1B
:10483000610E016F000E026F000E036F4FC104F195
:1048400050C105F151C106F152C107F155EC2FF0ED
:1048500003AF03D050EC30F01200C80E006FAF0E63
:10486000016F000E026F000E036F4FC104F150C1C3
:1048700005F151C106F152C107F166EC2FF01200AB
:104880000401730E826FCBEC0EF004012C0E826FCC
:10489000CBEC0EF0078462C166F163C167F164C1BD
:1048A00068F165C169F14BC14FF14CC150F14DC187
:1048B00051F14EC152F157C159F158C15AF1079403
:1048C00066EC24F0D5EC0EF084EF29F066C100F11F
:1048D00067C101F168C102F169C103F10101F3ECA3
:1048E0002FF0B6EC2DF00401630E826FCBEC0EF0CE
:1048F00004012C0E826FCBEC0EF04FC100F150C1C1
:1049000001F151C102F152C103F10101F3EC2FF0A9
:10491000B6EC2DF00401660E826FCBEC0EF00401B4
:104920002C0E826FCBEC0EF050EC30F059C100F140
:104930005AC101F10101F3EC2FF0B6EC2DF00401A6
:10494000740E826FCBEC0EF0120010820401530E35
:10495000826FCBEC0EF004012C0E826FCBEC0EF0CC
:1049600083C32AF184C32BF185C32CF186C32DF1B7
:1049700087C32EF188C32FF189C330F18AC331F187
:104980008BC332F18CC333F101019EEC30F015EC96
:1049900030F000C166F101C167F102C168F103C1E5
:1049A00069F18EC32AF18FC32BF190C32CF191C30F
:1049B0002DF192C32EF193C32FF194C330F195C31F
:1049C00031F196C332F197C333F101019EEC30F01F
:1049D00015EC30F000C14FF101C150F102C151F1AD
:1049E00003C152F191EC30F099C32FF19AC330F129
:1049F0009BC331F19CC332F19DC333F101019EECA5
:104A000030F015EC30F000C159F101C15AF166ECFB
:104A100024F004012C0E826FCBEC0EF020EF25F079
:104A2000118E1CA002D01CAE108C1BBE02D01BA489
:104A3000108E03018251520A02E10F8201D00F92BF
:104A40008251750A02E1108401D010948251550AF6
:104A500002E1108601D010968351310A03E11382DE
:104A6000138402D01392139403018351660A01E068
:104A700056D00401660E826FCBEC0EF004012C0EB2
:104A8000826FCBEC0EF05CEC23F0F3EC2FF02AC13C
:104A900082F40401300E8227CBEC0EF02BC182F49D
:104AA0000401300E8227CBEC0EF02CC182F40401FD
:104AB000300E8227CBEC0EF02DC182F40401300EB3
:104AC0008227CBEC0EF02EC182F40401300E822737
:104AD000CBEC0EF02FC182F40401300E8227CBEC18
:104AE0000EF030C182F40401300E8227CBEC0EF0C0
:104AF00031C182F40401300E8227CBEC0EF032C1BA
:104B000082F40401300E8227CBEC0EF033C182F424
:104B10000401300E8227CBEC0EF082EF29F011A0B9
:104B200003D011A401D01084078410B2F9EF25F04E
:104B300010A4DDEF25F0BAC166F1BBC167F1BCC1BD
:104B400068F1BDC169F1BEC16AF1BFC16BF1C0C1FD
:104B50006CF1C1C16DF1C2C16EF1C3C16FF1C4C1CD
:104B600070F1C5C171F1C6C172F1C7C173F1C8C19D
:104B700074F1C9C175F1CAC176F1CBC177F1CCC16D
:104B800078F1CDC179F1CEC17AF1CFC17BF1D0C13D
:104B90007CF1D1C17DF1D2C17EF1D3C17FF1D4C10D
:104BA00080F1D5C181F1D6C182F1D7C183F1D8C1DD
:104BB00084F1D9C185F1E5EF25F062C166F163C1E9
:104BC00067F164C168F165C169F1BAC186F1BBC121
:104BD00087F1BCC188F1BDC189F14BC14FF14CC116
:104BE00050F14DC151F14EC152F157C159F158C167
:104BF0005AF107940FA01BEF26F00101966708EF0A
:104C000026F0976708EF26F0986708EF26F0996777
:104C10000CEF26F01BEF26F05FEC22F096C104F1BA
:104C200097C105F198C106F199C107F155EC2FF034
:104C300003BF48EF29F05FEC22F00101000E046F82
:104C4000000E056F010E066F000E076F86EC2FF049
:104C500011A02AD011A228D0F3EC2FF0296701D09F
:104C600005D004012D0E826FCBEC0EF030C182F422
:104C70000401300E8227CBEC0EF031C182F4040126
:104C8000300E8227CBEC0EF032C182F40401300EDC
:104C90008227CBEC0EF033C182F40401300E822760
:104CA000CBEC0EF0D5EC0EF012A8C5D012981DC0BA
:104CB0001EF01E3A1E42070E1E1600011E50000A6C
:104CC000D8B4E7EF26F000011E50010AD8B473EF04
:104CD00026F000011E50020AD8B471EF26F019EF39
:104CE00027F019EF27F050EC30F02DC001F12EC065
:104CF00000F1D89001330033D89001330033010123
:104D0000630E046F000E056F000E066F000E076F36
:104D100086EC2FF0280E046F000E056F000E066F54
:104D2000000E076F55EC2FF000C130F050EC30F062
:104D30002BC001F1019F019D2CC000F10101A40EC7
:104D4000046F000E056F000E066F000E076F86ECF5
:104D50002FF000C12FF000C104F101C105F102C123
:104D600006F103C107F1640E006F000E016F000E23
:104D7000026F000E036F55EC2FF0050E046F000E4E
:104D8000056F000E066F000E076F86EC2FF000C156
:104D900004F101C105F102C106F103C107F150ECB4
:104DA00030F030C000F155EC2FF000C131F031C0CF
:104DB000E8FF050F305C03E78A8419EF27F031C064
:104DC000E8FF0A0F305C01E68A9419EF27F000C172
:104DD00024F101C125F102C126F103C127F150ECF4
:104DE00030F056EC30F01D501F0BE8CF00F1010100
:104DF000640E046F000E056F000E066F000E076F45
:104E000066EC2FF024C104F125C105F126C106F19D
:104E100027C107F155EC2FF003BF02D08A9401D0CF
:104E20008A8424C100F125C101F126C102F127C104
:104E300003F184EF29F000C124F101C125F102C181
:104E400026F103C127F110AE4DD0109E00C108F12C
:104E500001C109F102C10AF103C10BF1F3EC2FF01A
:104E600030C1E2F131C1E3F132C1E4F133C1E5F126
:104E700008C100F109C101F10AC102F10BC103F13E
:104E800001016C0E046F070E056F000E066F000E19
:104E9000076F55EC2FF003BF04D00101550EE66FEC
:104EA0001CD008C100F109C101F10AC102F10BC116
:104EB00003F10101A40E046F060E056F000E066FCC
:104EC000000E076F55EC2FF003BF04D001017F0ED9
:104ED000E66F03D00101FF0EE66F1F8E11AE48EFA3
:104EE00029F0119E24C100F125C101F126C102F172
:104EF00027C103F111A005D011A203D00FB048EFD4
:104F000029F010A48BEF27F00401750E826FCBEC13
:104F10000EF090EF27F00401720E826FCBEC0EF0D2
:104F200004012C0E826FCBEC0EF0F3EC2FF029670E
:104F30009FEF27F00401200E826FA2EF27F00401FB
:104F40002D0E826FCBEC0EF030C182F40401300ED6
:104F50008227CBEC0EF031C182F40401300E82279F
:104F6000CBEC0EF004012E0E826FCBEC0EF032C1B2
:104F700082F40401300E8227CBEC0EF033C182F4B0
:104F80000401300E8227CBEC0EF004016D0E826F0F
:104F9000CBEC0EF004012C0E826FCBEC0EF04FC167
:104FA00000F150C101F151C102F152C103F10101FF
:104FB000F3EC2FF0B6EC2DF00401480E826FCBEC31
:104FC0000EF004017A0E826FCBEC0EF004012C0E71
:104FD000826FCBEC0EF066C100F167C101F168C1D0
:104FE00002F169C103F10101F3EC2FF0B6EC2DF0F1
:104FF0000401630E826FCBEC0EF004012C0E826F65
:10500000CBEC0EF066C100F167C101F168C102F19D
:1050100069C103F101010A0E046F000E056F000E55
:10502000066F000E076F66EC2FF0000E046F120E75
:10503000056F000E066F000E076F86EC2FF0F3EC85
:105040002FF02AC182F40401300E8227CBEC0EF03F
:105050002BC182F40401300E8227CBEC0EF02CC160
:1050600082F40401300E8227CBEC0EF02DC182F4C5
:105070000401300E8227CBEC0EF02EC182F4040125
:10508000300E8227CBEC0EF02FC182F40401300EDB
:105090008227CBEC0EF030C182F40401300E82275F
:1050A000CBEC0EF004012E0E826FCBEC0EF031C172
:1050B00082F40401300E8227CBEC0EF032C182F470
:1050C0000401300E8227CBEC0EF033C182F40401D0
:1050D000300E8227CBEC0EF00401730E826FCBEC06
:1050E0000EF004012C0E826FCBEC0EF050EC30F081
:1050F00059C100F15AC101F1AEEC2AF013A2D0EF70
:1051000028F004012C0E826FCBEC0EF086C166F104
:1051100087C167F188C168F189C169F15FEC22F04C
:105120000101000E046F000E056F010E066F000EE8
:10513000076F86EC2FF0F3EC2FF02967A5EF28F02E
:105140000401200E826FA8EF28F004012D0E826F5B
:10515000CBEC0EF030C182F40401300E8227CBEC90
:105160000EF031C182F40401300E8227CBEC0EF038
:1051700004012E0E826FCBEC0EF032C182F40401DA
:10518000300E8227CBEC0EF033C182F40401300ED6
:105190008227CBEC0EF004016D0E826FCBEC0EF08B
:1051A00013A4F7EF28F004012C0E826FCBEC0EF065
:1051B00013ACE5EF28F00401500E826FCBEC0EF03B
:1051C000139C1398139AF7EF28F013AEF2EF28F020
:1051D0000401460E826FCBEC0EF0139E1398139AC7
:1051E000F7EF28F00401530E826FCBEC0EF038B0CD
:1051F0000EEF29F004012C0E826FCBEC0EF08BB079
:1052000009EF29F00401440E826FCBEC0EF00EEF93
:1052100029F00401530E826FCBEC0EF00FB214EFA5
:1052200029F00FA046EF29F004012C0E826FCBEC81
:105230000EF0200EF86EF76AF66A04010900F5CF49
:1052400082F4CBEC0EF00900F5CF82F4CBEC0EF03B
:105250000900F5CF82F4CBEC0EF00900F5CF82F413
:10526000CBEC0EF00900F5CF82F4CBEC0EF0090088
:10527000F5CF82F4CBEC0EF00900F5CF82F4CBEC45
:105280000EF00900F5CF82F4CBEC0EF0D5EC0EF069
:105290000F90109E129884EF29F00401630E826F24
:1052A000CBEC0EF004012C0E826FCBEC0EF08AECEE
:1052B00029F004012C0E826FCBEC0EF0FDEC29F0EE
:1052C00004012C0E826FCBEC0EF079EC2AF0040175
:1052D0002C0E826FCBEC0EF00101F80E006FCD0E9C
:1052E000016F660E026F030E036F9FEC29F004013D
:1052F0002C0E826FCBEC0EF08FEC2AF0D5EC0EF07A
:1053000084EF29F0D5EC0EF00301C26B07901092E8
:1053100093EF2CF0D8900E0E54EC0BF0E8CF00F188
:105320000F0E54EC0BF0E8CF01F1100E54EC0BF023
:10533000E8CF02F1110E54EC0BF0E8CF03F10101BC
:10534000000E046F000E056F010E066F000E076F52
:1053500086EC2FF0F3EC2FF02AC182F40401300E1A
:105360008227CBEC0EF02BC182F40401300E822791
:10537000CBEC0EF02CC182F40401300E8227CBEC72
:105380000EF02DC182F40401300E8227CBEC0EF01A
:105390002EC182F40401300E8227CBEC0EF02FC117
:1053A00082F40401300E8227CBEC0EF030C182F47F
:1053B0000401300E8227CBEC0EF031C182F40401DF
:1053C000300E8227CBEC0EF004012E0E826FCBEC58
:1053D0000EF032C182F40401300E8227CBEC0EF0C5
:1053E00033C182F40401300E8227CBEC0EF00401AD
:1053F0006D0E826FCBEC0EF01200120E54EC0BF01F
:10540000E8CF00F1130E54EC0BF0E8CF01F1140ECD
:1054100054EC0BF0E8CF02F1150E54EC0BF0E8CF92
:1054200003F101010A0E046F000E056F000E066FF6
:10543000000E076F66EC2FF0000E046F120E056F62
:10544000000E066F000E076F86EC2FF0F3EC2FF0C6
:105450002AC182F40401300E8227CBEC0EF02BC15E
:1054600082F40401300E8227CBEC0EF02CC182F4C2
:105470000401300E8227CBEC0EF02DC182F4040122
:10548000300E8227CBEC0EF02EC182F40401300ED8
:105490008227CBEC0EF02FC182F40401300E82275C
:1054A000CBEC0EF030C182F40401300E8227CBEC3D
:1054B0000EF004012E0E826FCBEC0EF031C182F49F
:1054C0000401300E8227CBEC0EF032C182F40401CD
:1054D000300E8227CBEC0EF033C182F40401300E83
:1054E0008227CBEC0EF00401730E826FCBEC0EF032
:1054F00012000A0E54EC0BF0E8CF00F10B0E54EC46
:105500000BF0E8CF01F10C0E54EC0BF0E8CF02F1F8
:105510000D0E54EC0BF0E8CF03F1AEEF2AF0060EBF
:1055200054EC0BF0E8CF00F1070E54EC0BF0E8CF91
:1055300001F1080E54EC0BF0E8CF02F1090E54EC27
:105540000BF0E8CF03F1AEEF2AF0010150EC30F0A0
:10555000078457C100F158C101F107940101E80E19
:10556000046F800E056F000E066F000E076F66EC6D
:105570002FF0000E046F040E056F000E066F000E74
:10558000076F86EC2FF0880E046F130E056F000E68
:10559000066F000E076F55EC2FF00A0E046F000E19
:1055A000056F000E066F000E076F86EC2FF0F3EC10
:1055B0002FF001012967E2EF2AF00401200E826F2B
:1055C000E5EF2AF004012D0E826FCBEC0EF030C116
:1055D00082F40401300E8227CBEC0EF031C182F44C
:1055E0000401300E8227CBEC0EF032C182F40401AC
:1055F000300E8227CBEC0EF004012E0E826FCBEC26
:105600000EF033C182F40401300E8227CBEC0EF091
:105610000401430E826FCBEC0EF0120087C32AF117
:1056200088C32BF189C32CF18AC32DF18BC32EF1D2
:105630008CC32FF18DC330F18EC331F190C332F1A1
:1056400091C333F10101296B9EEC30F015EC30F081
:105650000101000E046F000E056F010E066F000EB3
:10566000076F66EC2FF00E0E0C6E00C10BF03DECD8
:105670000BF00F0E0C6E01C10BF03DEC0BF0100E99
:105680000C6E02C10BF03DEC0BF0110E0C6E03C161
:105690000BF03DEC0BF004017A0E826FCBEC0EF0B8
:1056A00004012C0E826FCBEC0EF00401350E826FDC
:1056B000CBEC0EF004012C0E826FCBEC0EF08AECDA
:1056C00029F035EF22F087C32AF188C32BF189C373
:1056D0002CF18AC32DF18BC32EF18CC32FF18DC316
:1056E00030F18EC331F190C332F191C333F1010136
:1056F000296B9EEC30F015EC30F0880E046F130E21
:10570000056F000E066F000E076F5AEC2FF0000EAB
:10571000046F040E056F000E066F000E076F66EC37
:105720002FF00101E80E046F800E056F000E066F6A
:10573000000E076F86EC2FF00A0E0C6E00C10BF006
:105740003DEC0BF00B0E0C6E01C10BF03DEC0BF0C1
:105750000C0E0C6E02C10BF03DEC0BF00D0E0C6E3E
:1057600003C10BF03DEC0BF004017A0E826FCBEC21
:105770000EF004012C0E826FCBEC0EF00401360EFD
:10578000826FCBEC0EF004012C0E826FCBEC0EF08E
:1057900079EC2AF035EF22F087C32AF188C32BF188
:1057A00089C32CF18AC32DF18BC32EF18CC32FF149
:1057B0008DC330F18FC331F190C332F191C333F116
:1057C00001019EEC30F015EC30F0000E046F120E6B
:1057D000056F000E066F000E076F66EC2FF00101DB
:1057E0000A0E046F000E056F000E066F000E076FA5
:1057F00086EC2FF0120E0C6E00C10BF03DEC0BF09E
:10580000130E0C6E01C10BF03DEC0BF0140E0C6E80
:1058100002C10BF03DEC0BF0150E0C6E03C10BF04A
:105820003DEC0BF004017A0E826FCBEC0EF004011C
:105830002C0E826FCBEC0EF00401370E826FCBEC96
:105840000EF004012C0E826FCBEC0EF0FDEC29F073
:1058500035EF22F087C32AF188C32BF189C32CF1DD
:105860008AC32DF18BC32EF18CC32FF18DC330F180
:105870008EC331F190C332F191C333F10101296B31
:105880009EEC30F015EC30F0880E046F130E056FAF
:10589000000E066F000E076F5AEC2FF0000E046F1B
:1058A000040E056F000E066F000E076F66EC2FF0FA
:1058B0000101E80E046F800E056F000E066F000EEA
:1058C000076F86EC2FF0060E0C6E00C10BF03DEC5E
:1058D0000BF0070E0C6E01C10BF03DEC0BF0080E47
:1058E0000C6E02C10BF03DEC0BF0090E0C6E03C107
:1058F0000BF03DEC0BF004017A0E826FCBEC0EF056
:1059000004012C0E826FCBEC0EF00401380E826F76
:10591000CBEC0EF004012C0E826FCBEC0EF08FEC72
:105920002AF035EF22F007A806EF2DF00101800ED6
:10593000006F1A0E016F060E026F000E036F4BC14F
:1059400004F14CC105F14DC106F14EC107F155EC12
:105950002FF003BF4CEF2DF0B0EC2DF04BC100F158
:105960004CC101F14DC102F14EC103F1078262EC5D
:105970002EF018C104F119C105F11AC106F11BC1BD
:1059800007F1F80E006FCD0E016F660E026F030E69
:10599000036F55EC2FF00E0E0C6E00C10BF03DECBA
:1059A0000BF00F0E0C6E01C10BF03DEC0BF0100E66
:1059B0000C6E02C10BF03DEC0BF0110E0C6E03C12E
:1059C0000BF03DEC0BF00784010150EC30F057C1B7
:1059D00000F158C101F107940A0E0C6E00C10BF0E2
:1059E0003DEC0BF00B0E0C6E01C10BF03DEC0BF01F
:1059F0000C0E0C6E02C10BF03DEC0BF00D0E0C6E9C
:105A000003C10BF03DEC0BF04CEF2DF007AA4CEF6F
:105A10002DF00784010150EC30F057C100F158C15E
:105A200001F10794060E0C6E00C10BF03DEC0BF07B
:105A3000070E0C6E01C10BF03DEC0BF0080E0C6E66
:105A400002C10BF03DEC0BF0090E0C6E03C10BF024
:105A50003DEC0BF0078462C100F163C101F164C148
:105A600002F165C103F10794120E0C6E00C10BF038
:105A70003DEC0BF0130E0C6E01C10BF03DEC0BF086
:105A8000140E0C6E02C10BF03DEC0BF0150E0C6EFB
:105A900003C10BF03DEC0BF00798079A040180510D
:105AA00081197F0B0DE09EA8FED714EE00F0815106
:105AB0007F0BE126E750812B0F01AD6E4EEF2DF0ED
:105AC00005012F51010A0FE081AA78EF2DF00501A1
:105AD0002F51000AD8B49AEF37F000011650050A8A
:105AE000D8B49AEF37F081B878EF2DF099EC31F017
:105AF000F9EF0DF018C100F119C101F11AC102F15D
:105B00001BC103F1000E046F000E056F010E066F3E
:105B1000000E076F86EC2FF029A1A5EF2DF0205184
:105B2000D8B4A5EF2DF018C100F119C101F11AC1C7
:105B300002F11BC103F1000E046F000E056F0A0E87
:105B4000066F000E076F86EC2FF012000101045162
:105B500000130551011306510213075103131200DC
:105B60000101186B196B1A6B1B6B12002AC182F4AE
:105B70000401300E8227CBEC0EF02BC182F404011D
:105B8000300E8227CBEC0EF02CC182F40401300ED3
:105B90008227CBEC0EF02DC182F40401300E822757
:105BA000CBEC0EF02EC182F40401300E8227CBEC38
:105BB0000EF02FC182F40401300E8227CBEC0EF0E0
:105BC00030C182F40401300E8227CBEC0EF031C1DB
:105BD00082F40401300E8227CBEC0EF032C182F445
:105BE0000401300E8227CBEC0EF033C182F40401A5
:105BF000300E8227CBEC0EF012002FC182F404018C
:105C0000300E8227CBEC0EF030C182F40401300E4E
:105C10008227CBEC0EF031C182F40401300E8227D2
:105C2000CBEC0EF032C182F40401300E8227CBECB3
:105C30000EF033C182F40401300E8227CBEC0EF05B
:105C40001200060E216E060E226E060E236E212E07
:105C500027EF2EF0222E27EF2EF0232E27EF2EF007
:105C60008B84020E216E020E226E020E236E212EF6
:105C700037EF2EF0222E37EF2EF0232E37EF2EF0B7
:105C80008B941200FF0E226E22C023F0030E216EB1
:105C90008B84212E48EF2EF0030E216E232E48EF29
:105CA0002EF08B9422C023F0030E216E212E56EF8E
:105CB0002EF0030E216E233E56EF2EF0222E44EFDF
:105CC0002EF012000101005305E1015303E10253DC
:105CD00001E1002B25EC2FF050EC30F03951006F32
:105CE0003A51016F420E046F4B0E056F000E066FA6
:105CF000000E076F66EC2FF000C104F101C105F141
:105D000002C106F103C107F118C100F119C101F187
:105D10001AC102F11BC103F107B293EF2EF05AEC46
:105D20002FF095EF2EF055EC2FF000C118F101C1C6
:105D300019F102C11AF103C11BF1120050EC30F04D
:105D400059C100F15AC101F1060E54EC0BF0E8CF35
:105D500004F1070E54EC0BF0E8CF05F1080E54ECFB
:105D60000BF0E8CF06F1090E54EC0BF0E8CF07F189
:105D700055EC2FF000C124F101C125F102C126F13B
:105D800003C127F1290E046F000E056F000E066F88
:105D9000000E076F66EC2FF0EE0E046F430E056FDA
:105DA000000E066F000E076F5AEC2FF024C104F1AD
:105DB00025C105F126C106F127C107F166EC2FF0D8
:105DC00000C11CF101C11DF102C11EF103C11FF18F
:105DD000120E54EC0BF0E8CF04F1130E54EC0BF060
:105DE000E8CF05F1140E54EC0BF0E8CF06F1150ED8
:105DF00054EC0BF0E8CF07F10D0E006F000E016FB1
:105E0000000E026F000E036F66EC2FF0180E046F89
:105E1000000E056F000E066F000E076F86EC2FF068
:105E20001CC104F11DC105F11EC106F11FC107F11E
:105E30005AEC2FF06A0E046F2A0E056F000E066FE3
:105E4000000E076F55EC2FF01200BF0EFA6E200EF9
:105E50003A6F396BD8900037013702370337D8B023
:105E600036EF2FF03A2F2BEF2FF039073A07035375
:105E7000D8B412000331070B80093F6F03390F0BB1
:105E8000010F396F80EC5FF0406F390580EC5FF0F7
:105E9000405D405F396B3F33D8B0392739333FA974
:105EA0004BEF2FF0405139271200010175EC30F013
:105EB000D8B01200010103510719346F38EC30F0EB
:105EC000D8900751031934AF800F12000101346BD1
:105ED0005CEC30F0D8A072EC30F0D8B0120047EC97
:105EE00030F050EC30F01F0E366F88EC30F00B3590
:105EF000D8B038EC30F0D8A00335D8B01200362F27
:105F000075EF2FF034B15FEC30F012000101346B0B
:105F100004510511061107110008D8A05CEC30F0FF
:105F2000D8A072EC30F0D8B01200086B096B0A6B85
:105F30000B6B88EC30F01F0E366F88EC30F0075199
:105F40000B5DD8A4B0EF2FF006510A5DD8A4B0EFD6
:105F50002FF00551095DD8A4B0EF2FF00451085D72
:105F6000D8A0C3EF2FF00451085F0551D8A0053D1C
:105F7000095F0651D8A0063D0A5F0751D8A0073D2A
:105F80000B5FD8900081362F9DEF2FF034B15FEC7E
:105F900030F0346B5CEC30F0D8908CEC30F0075182
:105FA0000B5DD8A4E0EF2FF006510A5DD8A4E0EF16
:105FB0002FF00551095DD8A4E0EF2FF00451085DE2
:105FC000D8A0EFEF2FF0003FEFEF2FF0013FEFEF02
:105FD0002FF0023FEFEF2FF0032BD8B4120034B1B3
:105FE0005FEC30F012000101346B5CEC30F0D8B0A3
:105FF000120091EC30F0200E366F00370137023777
:10600000033711EE33F00A0E376FE7360A0EE75CFE
:10601000D8B0E76EE552372F05EF30F0362FFDEFA1
:106020002FF034B12981D890120001010A0E346F8B
:10603000200E366F11EE29F03451376F0A0ED890CA
:10604000E652D8B0E726E732372F20EF30F003339F
:10605000023301330033362F1AEF30F0E750FF0FD1
:10606000D8A00335D8B0120029B15FEC30F012008F
:10607000045100270551D8B0053D01270651D8B07D
:10608000063D02270751D8B0073D032712000051F3
:10609000086F0151096F02510A6F03510B6F120013
:1060A0000101006B016B026B036B12000101046BB9
:1060B000056B066B076B12000335D8A01200035165
:1060C000800B001F011F021F031F003F6FEF30F006
:1060D000013F6FEF30F0023F6FEF30F0032B342BB6
:1060E000032512000735D8A012000751800B041FAA
:1060F000051F061F071F043F85EF30F0053F85EFA2
:1061000030F0063F85EF30F0072B342B07251200C7
:106110000037013702370337083709370A370B379B
:1061200012000101296B2A6B2B6B2C6B2D6B2E6BD4
:106130002F6B306B316B326B336B120001012A51C4
:106140000F0B2A6F2B510F0B2B6F2C510F0B2C6F3A
:106150002D510F0B2D6F2E510F0B2E6F2F510F0B3B
:106160002F6F30510F0B306F31510F0B316F325198
:106170000F0B326F33510F0B336F120000C124F13C
:1061800001C125F102C126F103C127F104C100F1CB
:1061900005C101F106C102F107C103F124C104F1F7
:1061A00025C105F126C106F127C107F1120010A88B
:1061B00006D08994000EC76E220EC66E05D0898463
:1061C000000EC76E220EC66E050EE82EFED7120018
:1061D00010A802D0898401D08994050EE82EFED73C
:1061E0001200D7EC30F09E96C69E000EC96EFF0ED0
:1061F0009EB602D0E82EFCD79E96C69E000EC96EB3
:10620000FF0E9EB602D0E82EFCD7C9CFAFF59E9602
:10621000C69E000EC96EFF0E9EB602D0E82EFCD7B9
:10622000C9CFB0F59E96C69E000EC96EFF0E9EB6F3
:1062300002D0E82EFCD7C9CFB1F59E96C69E000EBF
:10624000C96EFF0E9EB602D0E82EFCD7C9CFB2F5BC
:106250009E96C69E000EC96EFF0E9EB602D0E82E18
:10626000FCD7C9CFB3F59E96C69E000EC96EFF0E31
:106270009EB602D0E82EFCD7C9CFB4F59E96C69E36
:10628000000EC96EFF0E9EB602D0E82EFCD7C9CF15
:10629000B5F5E8EC30F01200D7EC30F09E96C69ED3
:1062A000800EC96EFF0E9EB602D0E82EFCD79E96D9
:1062B000C69EAFC5C9FFFF0E9EB602D0E82EFCD722
:1062C0009E96C69EB0C5C9FFFF0E9EB602D0E82EB0
:1062D000FCD79E96C69EB1C5C9FFFF0E9EB602D0E2
:1062E000E82EFCD79E96C69EB2C5C9FFFF0E9EB68D
:1062F00002D0E82EFCD79E96C69EB3C5C9FFFF0EFE
:106300009EB602D0E82EFCD79E96C69EB4C5C9FFA5
:10631000FF0E9EB602D0E82EFCD79E96C69EB5C54F
:10632000C9FFFF0E9EB602D0E82EFCD7E8EC30F095
:106330001200D7EC30F09E96C69E070EC96EFF0E77
:106340009EB602D0E82EFCD79E96C69E000EC96E61
:10635000FF0E9EB602D0E82EFCD7C9CFAFF59E96B1
:10636000C69E000EC96EFF0E9EB602D0E82EFCD768
:10637000C9CFB0F59E96C69E000EC96EFF0E9EB6A2
:1063800002D0E82EFCD7C9CFB1F59E96C69E000E6E
:10639000C96EFF0E9EB602D0E82EFCD7C9CFB2F56B
:1063A000E8EC30F0D7EC30F09E96C69E25C0C9FFD1
:1063B000FF0E9EB602D0E82EFCD79E96C69E000E1B
:1063C000C96EFF0E9EB602D0E82EFCD7C9CFB6F537
:1063D000E8EC30F01200D7EC30F09E96C69E870EA7
:1063E000C96EFF0E9EB602D0E82EFCD79E96C69EC2
:1063F000AFC5C9FFFF0E9EB602D0E82EFCD79E9611
:10640000C69EB0C5C9FFFF0E9EB602D0E82EFCD7CF
:106410009E96C69EB1C5C9FFFF0E9EB602D0E82E5D
:10642000FCD79E96C69EB2C5C9FFFF0E9EB602D08F
:10643000E82EFCD7E8EC30F0D7EC30F09E96C69E04
:1064400026C0C9FFFF0E9EB602D0E82EFCD79E964E
:10645000C69EB6C5C9FFFF0E9EB602D0E82EFCD779
:10646000E8EC30F01200D7EC30F09E96C69E870E16
:10647000C96EFF0E9EB602D0E82EFCD79E96C69E31
:10648000000EC96EFF0E9EB602D0E82EFCD79E9677
:10649000C69E800EC96EFF0E9EB602D0E82EFCD7B7
:1064A0009E96C69E800EC96EFF0E9EB602D0E82E46
:1064B000FCD79E96C69E800EC96EFF0E9EB602D079
:1064C000E82EFCD7E8EC30F01200D7EC30F09E96C6
:1064D000C69E870EC96EFF0E9EB602D0E82EFCD770
:1064E0009E96C69E000EC96EFF0E9EB602D0E82E86
:1064F000FCD79E96C69E000EC96EFF0E9EB602D0B9
:10650000E82EFCD79E96C69E800EC96EFF0E9EB6E4
:1065100002D0E82EFCD79E96C69E800EC96EFF0E56
:106520009EB602D0E82EFCD7E8EC30F0120010A89E
:1065300017D0D7EC30F09E96C69E8F0EC96EFF0E18
:106540009EB602D0E82EFCD79E96C69E000EC96E5F
:10655000FF0E9EB602D0E82EFCD7E8EC30F0120019
:1065600099EC31F0120010A82DD0D7EC30F09E96A7
:10657000C69E26C0C9FFFF0E9EB602D0E82EFCD7ED
:106580009E96C69E450EC96EFF0E9EB602D0E82EA0
:10659000FCD7E8EC30F0D7EC30F09E96C69E8F0E1C
:1065A000C96EFF0E9EB602D0E82EFCD79E96C69E00
:1065B000000EC96EFF0E9EB602D0E82EFCD7E8ECA6
:1065C00030F01200D7EC30F09E96C69E26C0C9FF70
:1065D000FF0E9EB602D0E82EFCD79E96C69E010EF8
:1065E000C96EFF0E9EB602D0E82EFCD7E8EC30F064
:1065F000D7EC30F09E96C69E910EC96EFF0E9EB6E9
:1066000002D0E82EFCD79E96C69EA50EC96EFF0E40
:106610009EB602D0E82EFCD7E8EC30F01200D7ECA2
:1066200030F09E96C69E26C0C9FFFF0E9EB602D0D1
:10663000E82EFCD79E96C69E810EC96EFF0E9EB6B2
:1066400002D0E82EFCD7E8EC30F01200D7EC30F0A6
:106650009E96C69E26C0C9FFFF0E9EB602D0E82EAB
:10666000FCD79E96C69E010EC96EFF0E9EB602D046
:10667000E82EFCD7E8EC30F01200D7EC30F09E9614
:10668000C69E910EC96EFF0E9EB602D0E82EFCD7B4
:106690009E96C69EA50EC96EFF0E9EB602D0E82E2F
:1066A000FCD7E8EC30F01200D7EC30F09E96C69E96
:1066B000910EC96EFF0E9EB602D0E82EFCD79E96B4
:1066C000C69E000EC96EFF0E9EB602D0E82EFCD705
:1066D000E8EC30F012000501256B266B276B286B68
:1066E000899A400EC76E200EC66E9E96C69E030EF9
:1066F000C96EFF0E9EB602D0E82EFCD79E96C69EAF
:1067000027C5C9FFFF0E9EB602D0E82EFCD79E9685
:10671000C69E26C5C9FFFF0E9EB602D0E82EFCD746
:106720009E96C69E25C5C9FFFF0E9EB602D0E82ED6
:10673000FCD79E96C69EC952FF0E9EB602D0E82E8A
:10674000FCD7898A0F01C950FF0A01E11200050137
:106750002E51130A05E005012E51170A0CE0120014
:106760000501F00E256FFF0E266F0F0E276F000E2E
:10677000286FC4EF33F00501F00E256FFF0E266F72
:10678000FF0E276F000E286F899A400EC76E200EED
:10679000C66E9E96C69E030EC96EFF0E9EB602D0B2
:1067A000E82EFCD79E96C69E27C5C9FFFF0E9EB653
:1067B00002D0E82EFCD79E96C69E26C5C9FFFF0EC6
:1067C0009EB602D0E82EFCD79E96C69E25C5C9FF70
:1067D000FF0E9EB602D0E82EFCD79E96C69EC952EA
:1067E000FF0E9EB602D0E82EFCD7898A0F01C95051
:1067F000FF0A1DE005012E51130A05E005012E5187
:10680000170A0BE012000501000E256F000E266F1F
:10681000100E276F000E286F12000501000E256F65
:10682000000E266F000E276F010E286F1200050163
:10683000256B266B276B286B05012E51130A05E08B
:1068400005012E51170A0CE012000501000E216F00
:10685000000E226F080E236F000E246F39EF34F004
:106860000501000E216F000E226F800E236F000EB7
:10687000246F21C500F122C501F123C502F124C511
:1068800003F125C504F126C505F127C506F128C584
:1068900007F1A6EC2DF000C125F501C126F502C1D6
:1068A00027F503C128F5899A400EC76E200EC66EE3
:1068B0009E96C69E030EC96EFF0E9EB602D0E82EAF
:1068C000FCD79E96C69E27C5C9FFFF0E9EB602D076
:1068D000E82EFCD79E96C69E26C5C9FFFF0E9EB623
:1068E00002D0E82EFCD79E96C69E25C5C9FFFF0E96
:1068F0009EB602D0E82EFCD79E96C69EC952FF0EC9
:106900009EB602D0E82EFCD7898AC950FF0A08E15A
:1069100004C125F505C126F506C127F507C128F5EF
:10692000D890050124332333223321332151F00B36
:10693000216F05012167A4EF34F02267A4EF34F042
:106940002367A4EF34F0246739EF34F00501100E0B
:106950002527E86A2623E86A2723E86A2823120005
:10696000E86A05012E51130A06E005012E51170AA7
:106970000BE0020E120005012851000A03E1275125
:10698000F00B07E0010E120005012851000A01E09A
:10699000010E120029C500F12AC501F12BC502F133
:1069A0002CC503F125C504F126C505F127C506F15F
:1069B00028C507F155EC2FF003BF1200B0EC34F0FE
:1069C000D8A442EF35F0899A400EC76E200EC66EED
:1069D0009E96C69E060EC96EFF0E9EB602D0E82E8B
:1069E000FCD7898A899A9E96C69E020EC96EFF0EB2
:1069F0009EB602D0E82EFCD79E96C69E27C5C9FF3C
:106A0000FF0E9EB602D0E82EFCD79E96C69E26C5E7
:106A1000C9FFFF0E9EB602D0E82EFCD79E96C69EFA
:106A200025C5C9FFFF0E9EB602D0E82EFCD79E9664
:106A3000C69E000EC96EFF0E9EB602D0E82EFCD791
:106A4000898A899A9E96C69E050EC96EFF0E9EB6CD
:106A500002D0E82EFCD79E96C69EC952FF0E9EB667
:106A600002D0E82EFCD7C9B02BEF35F0898A05019A
:106A7000100E2527E86A2623E86A2723E86A2823D8
:106A8000CAEF34F01200899A400EC76E200EC66E0F
:106A90009E96C69E060EC96EFF0E9EB602D0E82ECA
:106AA000FCD7898A899A9E96C69EC70EC96EFF0E2C
:106AB0009EB602D0E82EFCD7898A0501256B266B8D
:106AC000276B286B1200899A400EC76E200EC66E87
:106AD0009E96C69E050EC96EFF0E9EB602D0E82E8B
:106AE000FCD79E96C69EC952FF0E9EB602D0E82ED7
:106AF000FCD7C9CF37F5898A1200899A400EC76E34
:106B0000200EC66E9E96C69EB90EC96EFF0E9EB62C
:106B100002D0E82EFCD7898A1200899A400EC76EEF
:106B2000200EC66E9E96C69EAB0EC96EFF0E9EB61A
:106B300002D0E82EFCD7898AFF0EE82EFED712007D
:106B4000B0EC34F0D8A41200899A400EC76E200E23
:106B5000C66E9E96C69E030EC96EFF0E9EB602D0EE
:106B6000E82EFCD79E96C69E27C5C9FFFF0E9EB68F
:106B700002D0E82EFCD79E96C69E26C5C9FFFF0E02
:106B80009EB602D0E82EFCD79E96C69E25C5C9FFAC
:106B9000FF0E9EB602D0E82EFCD79E96C69EC95226
:106BA000FF0E9EB602D0E82EFCD7898A0F01C9508D
:106BB000FF0AD8A40CEF37F00501FE0E376F37A09F
:106BC0003799F1EC30F0AFC538F5B0C539F5B1C53E
:106BD0003AF5B2C53BF5B3C53CF5B4C53DF5B5C511
:106BE0003EF50784BAC166F1BBC167F1BCC168F16B
:106BF000BDC169F14BC14FF14CC150F14DC151F1D3
:106C00004EC152F157C159F158C15AF10001165005
:106C1000010AD8B41AEF36F000011650020AD8B4AF
:106C20002BEF36F000011650040AD8B441EF36F0CD
:106C30000CEF37F00501000E466F8BA0379B5FEC21
:106C400022F000C13FF501C140F502C141F503C189
:106C500042F57AEF36F05FEC22F000C1DAF101C1C3
:106C6000DBF102C1DCF103C1DDF15CEC23F000C11A
:106C7000DEF101C1DFF102C1E0F103C1E1F10CEF8E
:106C800037F0379BDAC13FF5DBC140F5DCC141F598
:106C9000DDC142F55CEC23F0DEC104F1DFC105F19A
:106CA000E0C106F1E1C107F155EC2FF003AF5EEF53
:106CB00036F00501000E466F7AEF36F0720E046F63
:106CC000030E056F000E066F000E076F86EC2FF0A7
:106CD000036773EF36F0026773EF36F0016773EF07
:106CE00036F078EF36F00501FF0E466F7AEF36F09A
:106CF00000C146F50501616785EF36F0626785EFF3
:106D000036F0636785EF36F0646789EF36F09EEF03
:106D100036F0DAC100F1DBC101F1DCC102F1DDC105
:106D200003F161C504F162C505F163C506F164C5EF
:106D300007F155EC2FF003BF0CEF37F059C143F5C5
:106D40005AC144F5B9C545F50501110E326F899A4E
:106D5000400EC76E200EC66E9E96C69E060EC96E6B
:106D6000FF0E9EB602D0E82EFCD7898A899A9E969D
:106D7000C69E020EC96EFF0E9EB602D0E82EFCD74C
:106D80009E96C69E27C5C9FFFF0E9EB602D0E82E6E
:106D9000FCD79E96C69E26C5C9FFFF0E9EB602D0A2
:106DA000E82EFCD79E96C69E25C5C9FFFF0E9EB64F
:106DB00002D0E82EFCD725EE37F0322F02D0ECEFD0
:106DC00036F09E96C69EDECFC9FFFF0E9EB602D05D
:106DD000E82EFCD7DDEF36F0898A899A9E96C69E0A
:106DE000050EC96EFF0E9EB602D0E82EFCD79E9609
:106DF000C69EC952FF0E9EB602D0E82EFCD7C9B07F
:106E0000F7EF36F0898A0501100E2527E86A262358
:106E1000E86A2723E86A28230794120021C500F1B5
:106E200022C501F123C502F124C503F1899A400E60
:106E3000C76E200EC66E9E96C69E0B0EC96EFF0EC6
:106E40009EB602D0E82EFCD79E96C69E02C1C9FF10
:106E5000FF0E9EB602D0E82EFCD79E96C69E01C1BC
:106E6000C9FFFF0E9EB602D0E82EFCD79E96C69EA6
:106E700000C1C9FFFF0E9EB602D0E82EFCD79E9639
:106E8000C69EC952FF0E9EB602D0E82EFCD725EE54
:106E900037F00501100E326F9E96C69EC952FF0E46
:106EA0009EB602D0E82EFCD7C9CFDEFF322F4CEFC2
:106EB00037F0898A1200899A400EC76E200EC66E7E
:106EC0009E96C69E900EC96EFF0E9EB602D0E82E0C
:106ED000FCD79E96C69E000EC96EFF0E9EB602D0CF
:106EE000E82EFCD79E96C69E000EC96EFF0E9EB67B
:106EF00002D0E82EFCD79E96C69E000EC96EFF0EED
:106F00009EB602D0E82EFCD79E96C69EC952FF0EB2
:106F10009EB602D0E82EFCD7C9CF2DF59E96C69E10
:106F2000C952FF0E9EB602D0E82EFCD7C9CF2EF56F
:106F3000898A12008B9021EC2EF0B9C5E8FFD708A2
:106F400002E321EC2EF0B9C5E8FFC80802E321EC0A
:106F50002EF0B9C5E8FFB90802E321EC2EF0B9C55F
:106F6000E8FFAA0802E321EC2EF0B9C5E8FF9B0870
:106F700002E321EC2EF07DEC35F0F29CF29E8B9436
:106F8000C69AC2909482948C720ED36ED3A4FED70C
:106F900089968A909390F29AF2949D909E909D92F9
:106FA0009E92F298F29297EC32F0FF0EE8CF00F04A
:106FB000E82EFED7002EFCD7F290F286815081A8F1
:106FC000E4EF37F0F29E0300700ED36EF296F2906B
:0E6FD000010E376E038042EC2EF089EF0BF0BD
:10BF0000E844F926000C160C2B0C3F0C520C640C68
:10BF1000760C860C960CA50CB30CC10CCF0CDC0C6B
:06BF2000E80CF40C000C1B
:0200000400F00A
:0100C800FE39
:00000001FF
